 oal

 Timestamp is 4fb05c89 (Mon May 14 13:14:49 2012)

 Preferred load address is 00010000

 Start         Length     Name                   Class
 0001:00000000 00000194H .astart                 CODE
 0001:000001a0 00007460H .rdata                  CODE
 0001:00007600 00000020H .rdata$debug            CODE
 0001:00007620 0001378cH .text                   CODE
 0001:0001adac 00000050H .xdata                  CODE
 0001:0001adfc 00000000H .edata                  CODE
 0002:00000000 00006000H .KDATA                  DATA
 0003:00000000 000006b8H .data                   DATA
 0003:000006c0 00000a68H .bss                    DATA
 0004:00000000 00000820H .pdata                  DATA

  Address         Publics by Value              Rva+Base       Lib:Object

 0000:00000000       ___safe_se_handler_table   00000000     <absolute>
 0000:00000000       ___safe_se_handler_count   00000000     <absolute>
 0001:00000000       StartUp                    00011000 f   oal:startup.obj
 0001:000000f4       g_oalAddressTable          000110f4     oal:startup.obj
 0001:000001bc       pTOC                       000111bc     nkldr:ldrcmn.obj
 0001:000001c0       RomExt                     000111c0     nkldr:ldrcmn.obj
 0001:000001ec       ??_C@_0L@CPPPICDM@kernel?4dll?$AA@ 000111ec     nkldr:ldrcmn.obj
 0001:00000288       ??_C@_1BG@OFOAIMMC@?$AA?9?$AAO?$AAE?$AAM?$AAI?$AAn?$AAi?$AAt?$AA?$AN?$AA?6?$AA?$AA@ 00011288     oal:init.obj
 0001:000002a0       ??_C@_1EM@NOJFCDIG@?$AAE?$AAR?$AAR?$AAO?$AAR?$AA?3?$AA?5?$AAO?$AAE?$AAM?$AAI?$AAn?$AAi?$AAt?$AA?3?$AA?5?$AA?5?$AAS?$AAD?$AAM?$AAA?$AA?5?$AAn?$AAu?$AAl?$AAl?$AA?5?$AAp?$AAo?$AAi?$AAn?$AAt@ 000112a0     oal:init.obj
 0001:000002f0       ??_C@_1GI@LGFJGPEK@?$AAE?$AAR?$AAR?$AAO?$AAR?$AA?3?$AA?5?$AAO?$AAE?$AAM?$AAI?$AAn?$AAi?$AAt?$AA?3?$AA?5?$AAF?$AAa?$AAi?$AAl?$AAe?$AAd?$AA?5?$AAt?$AAo?$AA?5?$AAi?$AAn?$AAi?$AAt?$AAi?$AAa@ 000112f0     oal:init.obj
 0001:00000358       ??_C@_1GE@OIDINFAG@?$AAE?$AAR?$AAR?$AAO?$AAR?$AA?3?$AA?5?$AAO?$AAE?$AAM?$AAI?$AAn?$AAi?$AAt?$AA?3?$AA?5?$AAf?$AAa?$AAi?$AAl?$AAe?$AAd?$AA?5?$AAt?$AAo?$AA?5?$AAi?$AAn?$AAi?$AAt?$AAi?$AAa@ 00011358     oal:init.obj
 0001:000003bc       ??_C@_1DO@IDNOHJGN@?$AAO?$AAE?$AAM?$AAI?$AAn?$AAi?$AAt?$AA?3?$AA?5?$AA?5?$AAs?$AAi?$AAl?$AAi?$AAc?$AAo?$AAn?$AA?5?$AAr?$AAe?$AAv?$AA?5?$AA?$DN?$AA?5?$AA0?$AAx?$AA?$CF?$AAx?$AA?$AN?$AA?6?$AA?$AA@ 000113bc     oal:init.obj
 0001:000003fc       ??_C@_1DM@NOPJDCNN@?$AAO?$AAE?$AAM?$AAI?$AAn?$AAi?$AAt?$AA?3?$AA?5?$AA?5?$AAI?$AAI?$AAM?$AA?5?$AAn?$AAu?$AAl?$AAl?$AA?5?$AAp?$AAo?$AAi?$AAn?$AAt?$AAe?$AAr?$AA?$CB?$AA?$AN?$AA?6?$AA?$AA@ 000113fc     oal:init.obj
 0001:00000438       ??_C@_1EI@IDNMJAHA@?$AAR?$AAe?$AAs?$AAe?$AAt?$AA?5?$AAc?$AAa?$AAu?$AAs?$AAe?$AA?5?$AA?3?$AA?5?$AAU?$AAn?$AAk?$AAn?$AAo?$AAw?$AAn?$AA?5?$AAr?$AAe?$AAs?$AAe?$AAt?$AA?5?$AAc?$AAa?$AAu?$AAs@ 00011438     oal:init.obj
 0001:00000480       ??_C@_1DO@NKEBPIBC@?$AAR?$AAe?$AAs?$AAe?$AAt?$AA?5?$AAc?$AAa?$AAu?$AAs?$AAe?$AA?5?$AA?3?$AA?5?$AAW?$AAa?$AAt?$AAc?$AAh?$AAd?$AAo?$AAg?$AA?5?$AAR?$AAe?$AAs?$AAe?$AAt?$AA?$AN?$AA?6?$AA?$AA@ 00011480     oal:init.obj
 0001:000004c0       ??_C@_1DG@HBNDFBMN@?$AAR?$AAe?$AAs?$AAe?$AAt?$AA?5?$AAc?$AAa?$AAu?$AAs?$AAe?$AA?5?$AA?3?$AA?5?$AAJ?$AAT?$AAA?$AAG?$AA?5?$AAR?$AAe?$AAs?$AAe?$AAt?$AA?$AN?$AA?6?$AA?$AA@ 000114c0     oal:init.obj
 0001:000004f8       ??_C@_1DG@NKMOIPCI@?$AAR?$AAe?$AAs?$AAe?$AAt?$AA?5?$AAc?$AAa?$AAu?$AAs?$AAe?$AA?5?$AA?3?$AA?5?$AAS?$AAo?$AAf?$AAt?$AA?5?$AAR?$AAe?$AAs?$AAe?$AAt?$AA?$AN?$AA?6?$AA?$AA@ 000114f8     oal:init.obj
 0001:00000530       ??_C@_1DO@DFDJPBOH@?$AAR?$AAe?$AAs?$AAe?$AAt?$AA?5?$AAc?$AAa?$AAu?$AAs?$AAe?$AA?5?$AA?3?$AA?5?$AAR?$AAe?$AAs?$AAe?$AAt?$AA?5?$AAI?$AAn?$AA?5?$AAR?$AAe?$AAs?$AAe?$AAt?$AA?$AN?$AA?6?$AA?$AA@ 00011530     oal:init.obj
 0001:00000570       ??_C@_1DO@BLEAGBNL@?$AAR?$AAe?$AAs?$AAe?$AAt?$AA?5?$AAc?$AAa?$AAu?$AAs?$AAe?$AA?5?$AA?3?$AA?5?$AAP?$AAo?$AAw?$AAe?$AAr?$AA?5?$AAO?$AAn?$AA?5?$AAR?$AAe?$AAs?$AAe?$AAt?$AA?$AN?$AA?6?$AA?$AA@ 00011570     oal:init.obj
 0001:000005b0       ??_C@_1EI@BFFCEHAG@?$AA?5?$AA?5?$AA?5?$AA?5?$AA?5?$AA?5?$AA?5?$AAL?$AA1?$AAD?$AAS?$AAi?$AAz?$AAe?$AA?3?$AA?5?$AA?5?$AA?5?$AA?5?$AA?5?$AA?5?$AA?5?$AA0?$AAx?$AA?$CF?$AA0?$AA8?$AAx?$AA?5?$AA?$CI?$AA?$CF?$AAd@ 000115b0     oal:init.obj
 0001:000005f8       ??_C@_1EI@HCBBCEAB@?$AA?5?$AA?5?$AA?5?$AA?5?$AA?5?$AA?5?$AA?5?$AAL?$AA1?$AAD?$AAL?$AAi?$AAn?$AAe?$AAS?$AAi?$AAz?$AAe?$AA?3?$AA?5?$AA?5?$AA?5?$AA0?$AAx?$AA?$CF?$AA0?$AA8?$AAx?$AA?5?$AA?$CI?$AA?$CF?$AAd@ 000115f8     oal:init.obj
 0001:00000640       ??_C@_1EI@ODIOLNP@?$AA?5?$AA?5?$AA?5?$AA?5?$AA?5?$AA?5?$AA?5?$AAL?$AA1?$AAD?$AAN?$AAu?$AAm?$AAW?$AAa?$AAy?$AAs?$AA?3?$AA?5?$AA?5?$AA?5?$AA?5?$AA0?$AAx?$AA?$CF?$AA0?$AA8?$AAx?$AA?5?$AA?$CI?$AA?$CF?$AAd@ 00011640     oal:init.obj
 0001:00000688       ??_C@_1EI@MCDKAEIJ@?$AA?5?$AA?5?$AA?5?$AA?5?$AA?5?$AA?5?$AA?5?$AAL?$AA1?$AAD?$AAS?$AAe?$AAt?$AAs?$AAP?$AAe?$AAr?$AAW?$AAa?$AAy?$AA?3?$AA?5?$AA0?$AAx?$AA?$CF?$AA0?$AA8?$AAx?$AA?5?$AA?$CI?$AA?$CF?$AAd@ 00011688     oal:init.obj
 0001:000006d0       ??_C@_1EI@BPEMAFNI@?$AA?5?$AA?5?$AA?5?$AA?5?$AA?5?$AA?5?$AA?5?$AAL?$AA1?$AAI?$AAS?$AAi?$AAz?$AAe?$AA?3?$AA?5?$AA?5?$AA?5?$AA?5?$AA?5?$AA?5?$AA?5?$AA0?$AAx?$AA?$CF?$AA0?$AA8?$AAx?$AA?5?$AA?$CI?$AA?$CF?$AAd@ 000116d0     oal:init.obj
 0001:00000718       ??_C@_1EI@HIAPGGNP@?$AA?5?$AA?5?$AA?5?$AA?5?$AA?5?$AA?5?$AA?5?$AAL?$AA1?$AAI?$AAL?$AAi?$AAn?$AAe?$AAS?$AAi?$AAz?$AAe?$AA?3?$AA?5?$AA?5?$AA?5?$AA0?$AAx?$AA?$CF?$AA0?$AA8?$AAx?$AA?5?$AA?$CI?$AA?$CF?$AAd@ 00011718     oal:init.obj
 0001:00000760       ??_C@_1EI@ECGKJAB@?$AA?5?$AA?5?$AA?5?$AA?5?$AA?5?$AA?5?$AA?5?$AAL?$AA1?$AAI?$AAN?$AAu?$AAm?$AAW?$AAa?$AAy?$AAs?$AA?3?$AA?5?$AA?5?$AA?5?$AA?5?$AA0?$AAx?$AA?$CF?$AA0?$AA8?$AAx?$AA?5?$AA?$CI?$AA?$CF?$AAd@ 00011760     oal:init.obj
 0001:000007a8       ??_C@_1EI@MICEEGFH@?$AA?5?$AA?5?$AA?5?$AA?5?$AA?5?$AA?5?$AA?5?$AAL?$AA1?$AAI?$AAS?$AAe?$AAt?$AAs?$AAP?$AAe?$AAr?$AAW?$AAa?$AAy?$AA?3?$AA?5?$AA0?$AAx?$AA?$CF?$AA0?$AA8?$AAx?$AA?5?$AA?$CI?$AA?$CF?$AAd@ 000117a8     oal:init.obj
 0001:000007f0       ??_C@_1DO@CDJFGCON@?$AA?5?$AA?5?$AA?5?$AA?5?$AA?5?$AA?5?$AA?5?$AAL?$AA1?$AAF?$AAl?$AAa?$AAg?$AAs?$AA?3?$AA?5?$AA?5?$AA?5?$AA?5?$AA?5?$AA?5?$AA?5?$AA0?$AAx?$AA?$CF?$AA0?$AA8?$AAx?$AA?$AN?$AA?6?$AA?$AA@ 000117f0     oal:init.obj
 0001:00000830       ??_C@_1BI@NJKLHLEG@?$AA?5?$AA?5?$AA?5?$AAC?$AAa?$AAc?$AAh?$AAe?$AA?3?$AA?$AN?$AA?6?$AA?$AA@ 00011830     oal:init.obj
 0001:00000848       ??_C@_1BG@JHBBNGEC@?$AA?$CL?$AAO?$AAE?$AAM?$AAI?$AAn?$AAi?$AAt?$AA?$AN?$AA?6?$AA?$AA@ 00011848     oal:init.obj
 0001:000008f0       ??_C@_1EA@CDMGLANH@?$AAE?$AAR?$AAR?$AAO?$AAR?$AA?3?$AA?5?$AAF?$AAa?$AAi?$AAl?$AAe?$AAd?$AA?5?$AAt?$AAo?$AA?5?$AAR?$AAe?$AAa?$AAd?$AA?5?$AAR?$AAN?$AAG?$AAB?$AA?5?$AAI?$AAD?$AA?$AN?$AA?6?$AA?$AA@ 000118f0     oal:rngb.obj
 0001:00000930       ??_C@_1CK@MEEEGEFO@?$AAR?$AAN?$AAG?$AAB?$AA_?$AAG?$AAe?$AAt?$AAR?$AAa?$AAn?$AAd?$AAo?$AAm?$AAD?$AAa?$AAt?$AAa?$AA?$AN?$AA?6?$AA?$AA@ 00011930     oal:rngb.obj
 0001:00000a80       ??_C@_1FK@FNONLNGN@?$AA?$CF?$AAs?$AA?3?$AA?5?$AAD?$AAE?$AAB?$AAU?$AAG?$AAC?$AAH?$AAK?$AA?5?$AAf?$AAa?$AAi?$AAl?$AAe?$AAd?$AA?5?$AAi?$AAn?$AA?5?$AAf?$AAi?$AAl?$AAe?$AA?5?$AA?$CF?$AAs?$AA?5?$AAa@ 00011a80     oal:timer.obj
 0001:00000adc       ??_C@_1CO@EHGNHHJF@?$AAI?$AAn?$AAv?$AAa?$AAl?$AAi?$AAd?$AA?5?$AAT?$AAi?$AAm?$AAe?$AAr?$AA?5?$AAs?$AAo?$AAu?$AAr?$AAc?$AAe?$AA?$AN?$AA?6?$AA?$AA@ 00011adc     oal:timer.obj
 0001:00000b0c       ??_C@_1CI@OHCJFJPM@?$AAE?$AAR?$AAR?$AAO?$AAR?$AA?3?$AA?5?$AA?$CF?$AAs?$AA?5?$AAl?$AAi?$AAn?$AAe?$AA?5?$AA?$CF?$AAd?$AA?3?$AA?5?$AA?$AA@ 00011b0c     oal:timer.obj
 0001:00000b38       ??_C@_1IK@LIBHLIOI@?$AAC?$AA?3?$AA?2?$AAW?$AAI?$AAN?$AAC?$AAE?$AAR?$AAO?$AAO?$AAT?$AAS?$AA?2?$AAT?$AAo?$AAp?$AAa?$AAz?$AA?2?$AAW?$AAI?$AAN?$AAC?$AAE?$AA6?$AA0?$AA0?$AA?2?$AAP?$AAL?$AAA@ 00011b38     oal:timer.obj
 0001:00000bc8       ??_C@_1FE@CCLCEHKH@?$AAW?$AAd?$AAo?$AAg?$AAS?$AAe?$AAr?$AAv?$AAi?$AAc?$AAe?$AA?3?$AA?5?$AA?5?$AAW?$AAa?$AAt?$AAc?$AAh?$AAd?$AAo?$AAg?$AA?5?$AAn?$AAo?$AAt?$AA?5?$AAi?$AAn?$AAi?$AAt?$AAi@ 00011bc8     oal:timer.obj
 0001:00000c20       ??_C@_1EI@MHBJNECO@?$AAW?$AAd?$AAo?$AAg?$AAI?$AAn?$AAi?$AAt?$AA?3?$AA?5?$AA?5?$AAW?$AAa?$AAt?$AAc?$AAh?$AAd?$AAo?$AAg?$AA?5?$AAn?$AAu?$AAl?$AAl?$AA?5?$AAp?$AAo?$AAi?$AAn?$AAt?$AAe?$AAr@ 00011c20     oal:timer.obj
 0001:00000c68       ??_C@_1DA@GFBAMOOD@?$AA?9?$AAR?$AAe?$AAf?$AAr?$AAe?$AAs?$AAh?$AAW?$AAa?$AAt?$AAc?$AAh?$AAd?$AAo?$AAg?$AAT?$AAi?$AAm?$AAe?$AAr?$AA?$AN?$AA?6?$AA?$AA@ 00011c68     oal:timer.obj
 0001:00000c98       ??_C@_1KM@CBEKGBBP@?$AA?$CL?$AAR?$AAe?$AAf?$AAr?$AAe?$AAs?$AAh?$AAW?$AAa?$AAt?$AAc?$AAh?$AAd?$AAo?$AAg?$AAT?$AAi?$AAm?$AAe?$AAr?$AA?3?$AA?5?$AAS?$AAu?$AAb?$AAs?$AAe?$AAq?$AAu?$AAe?$AAn@ 00011c98     oal:timer.obj
 0001:00000d48       ??_C@_1JO@HOEBHJA@?$AA?$CL?$AAR?$AAe?$AAf?$AAr?$AAe?$AAs?$AAh?$AAW?$AAa?$AAt?$AAc?$AAh?$AAd?$AAo?$AAg?$AAT?$AAi?$AAm?$AAe?$AAr?$AA?3?$AA?5?$AAF?$AAi?$AAr?$AAs?$AAt?$AA?5?$AAc?$AAa?$AAl@ 00011d48     oal:timer.obj
 0001:00000de8       ??_C@_1DA@OILEKECL@?$AA?$CL?$AAR?$AAe?$AAf?$AAr?$AAe?$AAs?$AAh?$AAW?$AAa?$AAt?$AAc?$AAh?$AAd?$AAo?$AAg?$AAT?$AAi?$AAm?$AAe?$AAr?$AA?$AN?$AA?6?$AA?$AA@ 00011de8     oal:timer.obj
 0001:00000e18       ??_C@_1CK@OPIAODIP@?$AA?9?$AAI?$AAn?$AAi?$AAt?$AAW?$AAa?$AAt?$AAc?$AAh?$AAD?$AAo?$AAg?$AAT?$AAi?$AAm?$AAe?$AAr?$AA?$AN?$AA?6?$AA?$AA@ 00011e18     oal:timer.obj
 0001:00000e44       ??_C@_1CK@JPPHPFGJ@?$AA?$CL?$AAI?$AAn?$AAi?$AAt?$AAW?$AAa?$AAt?$AAc?$AAh?$AAD?$AAo?$AAg?$AAT?$AAi?$AAm?$AAe?$AAr?$AA?$AN?$AA?6?$AA?$AA@ 00011e44     oal:timer.obj
 0001:00000f00       ??_C@_1DC@BNLGCJKD@?$AA?9?$AAO?$AAA?$AAL?$AAT?$AAi?$AAm?$AAe?$AAr?$AAI?$AAn?$AAi?$AAt?$AA?$CI?$AAr?$AAc?$AA?5?$AA?$DN?$AA?5?$AA?$CF?$AAd?$AA?$CJ?$AA?$AN?$AA?6?$AA?$AA@ 00011f00     oal_timer_epit_common_topaz_v1:timer.obj
 0001:00000f38       ??_C@_1HM@CJGLDOPJ@?$AAE?$AAR?$AAR?$AAO?$AAR?$AA?3?$AA?5?$AAO?$AAA?$AAL?$AAT?$AAi?$AAm?$AAe?$AAr?$AAI?$AAn?$AAi?$AAt?$AA?3?$AA?5?$AAI?$AAn?$AAt?$AAe?$AAr?$AAr?$AAu?$AAp?$AAt?$AA?5?$AAe@ 00011f38     oal_timer_epit_common_topaz_v1:timer.obj
 0001:00000fb8       ??_C@_1EM@MOELPIPE@?$AA?$CL?$AAO?$AAA?$AAL?$AAT?$AAi?$AAm?$AAe?$AAr?$AAI?$AAn?$AAi?$AAt?$AA?3?$AA?5?$AA?5?$AAE?$AAP?$AAI?$AAT?$AA1?$AA?5?$AAn?$AAu?$AAl?$AAl?$AA?5?$AAp?$AAo?$AAi?$AAn?$AAt@ 00011fb8     oal_timer_epit_common_topaz_v1:timer.obj
 0001:00001008       ??_C@_1EI@OEMILFHD@?$AA?$CL?$AAO?$AAA?$AAL?$AAT?$AAi?$AAm?$AAe?$AAr?$AAI?$AAn?$AAi?$AAt?$AA?3?$AA?5?$AA?5?$AAS?$AAY?$AAS?$AAI?$AAN?$AAT?$AAR?$AA_?$AAU?$AAN?$AAD?$AAE?$AAF?$AAI?$AAN?$AAE@ 00012008     oal_timer_epit_common_topaz_v1:timer.obj
 0001:00001050       ??_C@_1HA@CPDFBGLD@?$AAE?$AAR?$AAR?$AAO?$AAR?$AA?3?$AA?5?$AAO?$AAA?$AAL?$AAT?$AAi?$AAm?$AAe?$AAr?$AAI?$AAn?$AAi?$AAt?$AA?3?$AA?5?$AAS?$AAy?$AAs?$AAt?$AAe?$AAm?$AA?5?$AAt?$AAi?$AAc?$AAk@ 00012050     oal_timer_epit_common_topaz_v1:timer.obj
 0001:000010c0       ??_C@_1KC@OOPLMPBN@?$AAE?$AAR?$AAR?$AAO?$AAR?$AA?3?$AA?5?$AAO?$AAA?$AAL?$AAT?$AAi?$AAm?$AAe?$AAr?$AAI?$AAn?$AAi?$AAt?$AA?3?$AA?5?$AAS?$AAy?$AAs?$AAt?$AAe?$AAm?$AA?5?$AAt?$AAi?$AAc?$AAk@ 000120c0     oal_timer_epit_common_topaz_v1:timer.obj
 0001:00001168       ??_C@_1GG@GKKJLMHA@?$AAO?$AAA?$AAL?$AAT?$AAi?$AAm?$AAe?$AAr?$AAI?$AAn?$AAi?$AAt?$AA?3?$AA?5?$AA?5?$AA3?$AA2?$AA7?$AA6?$AA8?$AA?5?$AAH?$AAz?$AA?5?$AAC?$AAK?$AAI?$AAL?$AA?5?$AAs?$AAu?$AAp@ 00012168     oal_timer_epit_common_topaz_v1:timer.obj
 0001:000011d0       ??_C@_1DM@HOCGOKJC@?$AA?$CL?$AAO?$AAA?$AAL?$AAT?$AAi?$AAm?$AAe?$AAr?$AAI?$AAn?$AAi?$AAt?$AA?$CI?$AA?5?$AA?$CF?$AAd?$AA?0?$AA?5?$AA?$CF?$AAd?$AA?0?$AA?5?$AA?$CF?$AAd?$AA?5?$AA?$CJ?$AA?$AN?$AA?6?$AA?$AA@ 000121d0     oal_timer_epit_common_topaz_v1:timer.obj
 0001:000012a0       ??_C@_1DA@OJCJANFP@?$AA?9?$AAO?$AAA?$AAL?$AAI?$AAn?$AAt?$AAr?$AAI?$AAn?$AAi?$AAt?$AA?$CI?$AAr?$AAc?$AA?5?$AA?$DN?$AA?5?$AA?$CF?$AAd?$AA?$CJ?$AA?$AN?$AA?6?$AA?$AA@ 000122a0     oal_intr_mx25_topaz_v1:intr.obj
 0001:000012d0       ??_C@_1EK@MEJGPAJO@?$AAO?$AAA?$AAL?$AAI?$AAn?$AAt?$AAr?$AAI?$AAn?$AAi?$AAt?$AA?3?$AA?5?$AAc?$AAa?$AAn?$AA?8?$AAt?$AA?5?$AAe?$AAn?$AAa?$AAb?$AAl?$AAe?$AA?5?$AAI?$AAR?$AAQ?$AA_?$AAS?$AAD@ 000122d0     oal_intr_mx25_topaz_v1:intr.obj
 0001:00001320       ??_C@_1EE@LFGNAGIB@?$AAO?$AAA?$AAL?$AAI?$AAn?$AAt?$AAr?$AAI?$AAn?$AAi?$AAt?$AA?3?$AA?5?$AAS?$AAD?$AAM?$AAA?$AA?5?$AAn?$AAu?$AAl?$AAl?$AA?5?$AAp?$AAo?$AAi?$AAn?$AAt?$AAe?$AAr?$AA?$CB?$AA?$AN@ 00012320     oal_intr_mx25_topaz_v1:intr.obj
 0001:00001368       ??_C@_1EG@GPGMOAIM@?$AAO?$AAA?$AAL?$AAI?$AAn?$AAt?$AAr?$AAI?$AAn?$AAi?$AAt?$AA?3?$AA?5?$AAG?$AAP?$AAI?$AAO?$AA4?$AA?5?$AAn?$AAu?$AAl?$AAl?$AA?5?$AAp?$AAo?$AAi?$AAn?$AAt?$AAe?$AAr?$AA?$CB@ 00012368     oal_intr_mx25_topaz_v1:intr.obj
 0001:000013b0       ??_C@_1EG@DDNMMDOF@?$AAO?$AAA?$AAL?$AAI?$AAn?$AAt?$AAr?$AAI?$AAn?$AAi?$AAt?$AA?3?$AA?5?$AAG?$AAP?$AAI?$AAO?$AA3?$AA?5?$AAn?$AAu?$AAl?$AAl?$AA?5?$AAp?$AAo?$AAi?$AAn?$AAt?$AAe?$AAr?$AA?$CB@ 000123b0     oal_intr_mx25_topaz_v1:intr.obj
 0001:000013f8       ??_C@_1EG@KGKMBHHA@?$AAO?$AAA?$AAL?$AAI?$AAn?$AAt?$AAr?$AAI?$AAn?$AAi?$AAt?$AA?3?$AA?5?$AAG?$AAP?$AAI?$AAO?$AA2?$AA?5?$AAn?$AAu?$AAl?$AAl?$AA?5?$AAp?$AAo?$AAi?$AAn?$AAt?$AAe?$AAr?$AA?$CB@ 000123f8     oal_intr_mx25_topaz_v1:intr.obj
 0001:00001440       ??_C@_1EG@MCEMGMIO@?$AAO?$AAA?$AAL?$AAI?$AAn?$AAt?$AAr?$AAI?$AAn?$AAi?$AAt?$AA?3?$AA?5?$AAG?$AAP?$AAI?$AAO?$AA1?$AA?5?$AAn?$AAu?$AAl?$AAl?$AA?5?$AAp?$AAo?$AAi?$AAn?$AAt?$AAe?$AAr?$AA?$CB@ 00012440     oal_intr_mx25_topaz_v1:intr.obj
 0001:00001488       ??_C@_1EE@OEGGBDGD@?$AAO?$AAA?$AAL?$AAI?$AAn?$AAt?$AAr?$AAI?$AAn?$AAi?$AAt?$AA?3?$AA?5?$AAA?$AAV?$AAI?$AAC?$AA?5?$AAn?$AAu?$AAl?$AAl?$AA?5?$AAp?$AAo?$AAi?$AAn?$AAt?$AAe?$AAr?$AA?$CB?$AA?$AN@ 00012488     oal_intr_mx25_topaz_v1:intr.obj
 0001:000014cc       ??_C@_1BO@IIKFLMMI@?$AA?$CL?$AAO?$AAA?$AAL?$AAI?$AAn?$AAt?$AAr?$AAI?$AAn?$AAi?$AAt?$AA?$AN?$AA?6?$AA?$AA@ 000124cc     oal_intr_mx25_topaz_v1:intr.obj
 0001:000014ec       ??_C@_1DO@NDIEKHNP@?$AA?9?$AAO?$AAA?$AAL?$AAI?$AAn?$AAt?$AAr?$AAR?$AAe?$AAq?$AAu?$AAe?$AAs?$AAt?$AAI?$AAr?$AAq?$AAs?$AA?$CI?$AAr?$AAc?$AA?5?$AA?$DN?$AA?5?$AA?$CF?$AAd?$AA?$CJ?$AA?$AN?$AA?6?$AA?$AA@ 000124ec     oal_intr_mx25_topaz_v1:intr.obj
 0001:00001530       ??_C@_1HO@EBPJKEJJ@?$AA?$CL?$AAO?$AAA?$AAL?$AAI?$AAn?$AAt?$AAr?$AAR?$AAe?$AAq?$AAu?$AAe?$AAs?$AAt?$AAI?$AAr?$AAq?$AAs?$AA?$CI?$AA0?$AAx?$AA?$CF?$AA0?$AA8?$AAx?$AA?9?$AA?$DO?$AA?$CF?$AAd?$AA?1?$AA?$CF@ 00012530     oal_intr_mx25_topaz_v1:intr.obj
 0001:000015b0       ??_C@_1DM@INNHDHDJ@?$AA?9?$AAO?$AAA?$AAL?$AAI?$AAn?$AAt?$AAr?$AAE?$AAn?$AAa?$AAb?$AAl?$AAe?$AAI?$AAr?$AAq?$AAs?$AA?$CI?$AAr?$AAc?$AA?5?$AA?$DN?$AA?5?$AA?$CF?$AAd?$AA?$CJ?$AA?$AN?$AA?6?$AA?$AA@ 000125b0     oal_intr_mx25_topaz_v1:intr.obj
 0001:000015f0       ??_C@_1EC@MDFPIGAB@?$AA?$CL?$AAO?$AAA?$AAL?$AAI?$AAn?$AAt?$AAr?$AAE?$AAn?$AAa?$AAb?$AAl?$AAe?$AAI?$AAr?$AAq?$AAs?$AA?$CI?$AA?$CF?$AAd?$AA?0?$AA?5?$AA0?$AAx?$AA?$CF?$AA0?$AA8?$AAx?$AA?$CJ?$AA?$AN?$AA?6@ 000125f0     oal_intr_mx25_topaz_v1:intr.obj
 0001:00001634       ??_C@_1CM@GPENGBBP@?$AA?9?$AAO?$AAA?$AAL?$AAI?$AAn?$AAt?$AAr?$AAD?$AAi?$AAs?$AAa?$AAb?$AAl?$AAe?$AAI?$AAr?$AAq?$AAs?$AA?$AN?$AA?6?$AA?$AA@ 00012634     oal_intr_mx25_topaz_v1:intr.obj
 0001:00001660       ??_C@_1EE@NIPMEMC@?$AA?$CL?$AAO?$AAA?$AAL?$AAI?$AAn?$AAt?$AAr?$AAD?$AAi?$AAs?$AAa?$AAb?$AAl?$AAe?$AAI?$AAr?$AAq?$AAs?$AA?$CI?$AA?$CF?$AAd?$AA?0?$AA?5?$AA0?$AAx?$AA?$CF?$AA0?$AA8?$AAx?$AA?$CJ?$AA?$AN@ 00012660     oal_intr_mx25_topaz_v1:intr.obj
 0001:000016a4       ??_C@_1CG@LBOJEJPE@?$AA?9?$AAO?$AAA?$AAL?$AAI?$AAn?$AAt?$AAr?$AAD?$AAo?$AAn?$AAe?$AAI?$AAr?$AAq?$AAs?$AA?$AN?$AA?6?$AA?$AA@ 000126a4     oal_intr_mx25_topaz_v1:intr.obj
 0001:000016cc       ??_C@_1DO@FCJPHKGC@?$AA?$CL?$AAO?$AAA?$AAL?$AAI?$AAn?$AAt?$AAr?$AAD?$AAo?$AAn?$AAe?$AAI?$AAr?$AAq?$AAs?$AA?$CI?$AA?$CF?$AAd?$AA?0?$AA?5?$AA0?$AAx?$AA?$CF?$AA0?$AA8?$AAx?$AA?$CJ?$AA?$AN?$AA?6?$AA?$AA@ 000126cc     oal_intr_mx25_topaz_v1:intr.obj
 0001:00001710       ??_C@_1FI@JHAKENKF@?$AAO?$AAE?$AAM?$AAI?$AAn?$AAt?$AAe?$AAr?$AAr?$AAu?$AAp?$AAt?$AAH?$AAa?$AAn?$AAd?$AAl?$AAe?$AAr?$AA?3?$AA?5?$AA?5?$AAu?$AAn?$AAd?$AAe?$AAf?$AAi?$AAn?$AAe?$AAd?$AA?5@ 00012710     oal_intr_mx25_topaz_v1:intr.obj
 0001:00001768       ??_C@_1FK@NCAAMDDH@?$AAO?$AAE?$AAM?$AAI?$AAn?$AAt?$AAe?$AAr?$AAr?$AAu?$AAp?$AAH?$AAa?$AAn?$AAd?$AAl?$AAe?$AAr?$AA?3?$AA?5?$AA?5?$AAN?$AAo?$AA?5?$AAp?$AAe?$AAn?$AAd?$AAi?$AAn?$AAg?$AA?5@ 00012768     oal_intr_mx25_topaz_v1:intr.obj
 0001:00001858       ??_C@_1CE@HFBIALPK@?$AA?9?$AAO?$AAA?$AAL?$AAI?$AAn?$AAt?$AAr?$AAM?$AAa?$AAp?$AAI?$AAn?$AAi?$AAt?$AA?$AN?$AA?6?$AA?$AA@ 00012858     oal_intr_mx25_topaz_v1:map.obj
 0001:0000187c       ??_C@_1CE@LMNIPMAG@?$AA?$CL?$AAO?$AAA?$AAL?$AAI?$AAn?$AAt?$AAr?$AAM?$AAa?$AAp?$AAI?$AAn?$AAi?$AAt?$AA?$AN?$AA?6?$AA?$AA@ 0001287c     oal_intr_mx25_topaz_v1:map.obj
 0001:000018a0       ??_C@_1DE@CBLJKBBB@?$AA?9?$AAO?$AAA?$AAL?$AAI?$AAn?$AAt?$AAr?$AAS?$AAt?$AAa?$AAt?$AAi?$AAc?$AAT?$AAr?$AAa?$AAn?$AAs?$AAl?$AAa?$AAt?$AAe?$AA?$AN?$AA?6?$AA?$AA@ 000128a0     oal_intr_mx25_topaz_v1:map.obj
 0001:000018d8       ??_C@_1EE@DPKCCBO@?$AA?$CL?$AAO?$AAA?$AAL?$AAI?$AAn?$AAt?$AAr?$AAS?$AAt?$AAa?$AAt?$AAi?$AAc?$AAT?$AAr?$AAa?$AAn?$AAs?$AAl?$AAa?$AAt?$AAe?$AA?$CI?$AA?$CF?$AAd?$AA?0?$AA?5?$AA?$CF?$AAd?$AA?$CJ?$AA?$AN@ 000128d8     oal_intr_mx25_topaz_v1:map.obj
 0001:00001920       ??_C@_1EA@JDMBMDEN@?$AA?9?$AAO?$AAA?$AAL?$AAT?$AAr?$AAa?$AAn?$AAs?$AAl?$AAa?$AAt?$AAe?$AAS?$AAy?$AAs?$AAI?$AAn?$AAt?$AAr?$AA?$CI?$AAr?$AAc?$AA?5?$AA?$DN?$AA?5?$AA?$CF?$AAd?$AA?$CJ?$AA?$AN?$AA?6?$AA?$AA@ 00012920     oal_intr_mx25_topaz_v1:map.obj
 0001:00001960       ??_C@_1DG@HAMHNOBJ@?$AA?$CL?$AAO?$AAA?$AAL?$AAT?$AAr?$AAa?$AAn?$AAs?$AAl?$AAa?$AAt?$AAe?$AAS?$AAy?$AAs?$AAI?$AAn?$AAt?$AAr?$AA?$CI?$AA?$CF?$AAd?$AA?$CJ?$AA?$AN?$AA?6?$AA?$AA@ 00012960     oal_intr_mx25_topaz_v1:map.obj
 0001:00001998       ??_C@_1EK@JOJPHPGP@?$AA?9?$AAO?$AAA?$AAL?$AAI?$AAn?$AAt?$AAr?$AAT?$AAr?$AAa?$AAn?$AAs?$AAl?$AAa?$AAt?$AAe?$AAI?$AAr?$AAq?$AA?$CI?$AAs?$AAy?$AAs?$AAI?$AAn?$AAt?$AAr?$AA?5?$AA?$DN?$AA?5?$AA?$CF@ 00012998     oal_intr_mx25_topaz_v1:map.obj
 0001:000019e4       ??_C@_1DG@IAFKCJEB@?$AA?$CL?$AAO?$AAA?$AAL?$AAI?$AAn?$AAt?$AAr?$AAT?$AAr?$AAa?$AAn?$AAs?$AAl?$AAa?$AAt?$AAe?$AAI?$AAr?$AAq?$AA?$CI?$AA?$CF?$AAd?$AA?$CJ?$AA?$AN?$AA?6?$AA?$AA@ 000129e4     oal_intr_mx25_topaz_v1:map.obj
 0001:00001a20       ??_C@_1EO@CCPDBEFN@?$AA?9?$AAO?$AAA?$AAL?$AAI?$AAn?$AAt?$AAr?$AAR?$AAe?$AAq?$AAu?$AAe?$AAs?$AAt?$AAS?$AAy?$AAs?$AAI?$AAn?$AAt?$AAr?$AA?$CI?$AAs?$AAy?$AAs?$AAI?$AAn?$AAt?$AAr?$AA?5?$AA?$DN@ 00012a20     oal_intr_mx25_topaz_v1:map.obj
 0001:00001a70       ??_C@_1HG@GANLJKGD@?$AAE?$AAR?$AAR?$AAO?$AAR?$AA?3?$AA?5?$AAO?$AAA?$AAL?$AAI?$AAn?$AAt?$AAr?$AAR?$AAe?$AAq?$AAu?$AAe?$AAs?$AAt?$AAS?$AAy?$AAs?$AAI?$AAn?$AAt?$AAr?$AA?3?$AA?5?$AAN?$AAo@ 00012a70     oal_intr_mx25_topaz_v1:map.obj
 0001:00001ae8       ??_C@_1JG@CKDDKDGB@?$AAE?$AAR?$AAR?$AAO?$AAR?$AA?3?$AA?5?$AAO?$AAA?$AAL?$AAI?$AAn?$AAt?$AAr?$AAR?$AAe?$AAq?$AAu?$AAe?$AAs?$AAt?$AAS?$AAy?$AAs?$AAI?$AAn?$AAt?$AAr?$AA?3?$AA?5?$AAS?$AAt@ 00012ae8     oal_intr_mx25_topaz_v1:map.obj
 0001:00001b80       ??_C@_1GI@NODFOAGP@?$AAE?$AAR?$AAR?$AAO?$AAR?$AA?3?$AA?5?$AAO?$AAA?$AAL?$AAI?$AAn?$AAt?$AAr?$AAR?$AAe?$AAq?$AAu?$AAe?$AAs?$AAt?$AAS?$AAy?$AAs?$AAI?$AAn?$AAt?$AAr?$AA?3?$AA?5?$AAI?$AAR@ 00012b80     oal_intr_mx25_topaz_v1:map.obj
 0001:00001be8       ??_C@_1IM@ENJFJBNJ@?$AAE?$AAR?$AAR?$AAO?$AAR?$AA?3?$AA?5?$AAO?$AAA?$AAL?$AAI?$AAn?$AAt?$AAr?$AAR?$AAe?$AAq?$AAu?$AAe?$AAs?$AAt?$AAS?$AAy?$AAs?$AAI?$AAn?$AAt?$AAr?$AA?3?$AA?5?$AAO?$AAn@ 00012be8     oal_intr_mx25_topaz_v1:map.obj
 0001:00001c78       ??_C@_1FK@JNHCPMAP@?$AA?$CL?$AAO?$AAA?$AAL?$AAI?$AAn?$AAt?$AAr?$AAR?$AAe?$AAq?$AAu?$AAe?$AAs?$AAt?$AAS?$AAy?$AAs?$AAI?$AAn?$AAt?$AAr?$AA?$CI?$AA?$CF?$AAd?$AA?0?$AA?5?$AA0?$AAx?$AA?$CF?$AA0?$AA8@ 00012c78     oal_intr_mx25_topaz_v1:map.obj
 0001:00001cd8       ??_C@_1EE@GBADJBKJ@?$AA?9?$AAO?$AAA?$AAL?$AAI?$AAn?$AAt?$AAr?$AAR?$AAe?$AAl?$AAe?$AAa?$AAs?$AAe?$AAS?$AAy?$AAs?$AAI?$AAn?$AAt?$AAr?$AA?$CI?$AAr?$AAc?$AA?5?$AA?$DN?$AA?5?$AA?$CF?$AAd?$AA?$CJ?$AA?$AN@ 00012cd8     oal_intr_mx25_topaz_v1:map.obj
 0001:00001d20       ??_C@_1HC@BIEMDHNG@?$AAE?$AAR?$AAR?$AAO?$AAR?$AA?3?$AA?5?$AAO?$AAA?$AAL?$AAI?$AAn?$AAt?$AAr?$AAR?$AAe?$AAl?$AAe?$AAa?$AAs?$AAe?$AAS?$AAy?$AAs?$AAI?$AAn?$AAt?$AAr?$AA?3?$AA?5?$AAI?$AAn@ 00012d20     oal_intr_mx25_topaz_v1:map.obj
 0001:00001d94       ??_C@_1DK@GDEEGDPM@?$AA?$CL?$AAO?$AAA?$AAL?$AAI?$AAn?$AAt?$AAr?$AAR?$AAe?$AAl?$AAe?$AAa?$AAs?$AAe?$AAS?$AAy?$AAs?$AAI?$AAn?$AAt?$AAr?$AA?$CI?$AA?$CF?$AAd?$AA?$CJ?$AA?$AN?$AA?6?$AA?$AA@ 00012d94     oal_intr_mx25_topaz_v1:map.obj
 0001:00001dd0       ??_C@_1DM@KHBFOEPK@?$AA?9?$AAO?$AAE?$AAM?$AAI?$AAn?$AAt?$AAe?$AAr?$AAr?$AAu?$AAp?$AAt?$AAE?$AAn?$AAa?$AAb?$AAl?$AAe?$AA?$CI?$AAr?$AAc?$AA?5?$AA?$DN?$AA?5?$AA1?$AA?$CJ?$AA?$AN?$AA?6?$AA?$AA@ 00012dd0     oal_intr_mx25_topaz_v1:map.obj
 0001:00001e10       ??_C@_1GM@HBOEKNIJ@?$AAE?$AAR?$AAR?$AAO?$AAR?$AA?3?$AA?5?$AAO?$AAE?$AAM?$AAI?$AAn?$AAt?$AAe?$AAr?$AAr?$AAu?$AAp?$AAt?$AAE?$AAn?$AAa?$AAb?$AAl?$AAe?$AA?3?$AA?5?$AAI?$AAn?$AAv?$AAa?$AAl@ 00012e10     oal_intr_mx25_topaz_v1:map.obj
 0001:00001e80       ??_C@_1EI@HHGIJMMI@?$AA?$CL?$AAO?$AAE?$AAM?$AAI?$AAn?$AAt?$AAe?$AAr?$AAr?$AAu?$AAp?$AAt?$AAE?$AAn?$AAa?$AAb?$AAl?$AAe?$AA?$CI?$AA?$CF?$AAd?$AA?0?$AA?5?$AA0?$AAx?$AA?$CF?$AAx?$AA?0?$AA?5?$AA?$CF?$AAd@ 00012e80     oal_intr_mx25_topaz_v1:map.obj
 0001:00001ec8       ??_C@_1CO@FKOPLHGO@?$AA?9?$AAO?$AAE?$AAM?$AAI?$AAn?$AAt?$AAe?$AAr?$AAr?$AAu?$AAp?$AAt?$AAD?$AAi?$AAs?$AAa?$AAb?$AAl?$AAe?$AA?$AN?$AA?6?$AA?$AA@ 00012ec8     oal_intr_mx25_topaz_v1:map.obj
 0001:00001ef8       ??_C@_1GO@FAMMIFAH@?$AAE?$AAR?$AAR?$AAO?$AAR?$AA?3?$AA?5?$AAO?$AAE?$AAM?$AAI?$AAn?$AAt?$AAe?$AAr?$AAr?$AAu?$AAp?$AAt?$AAD?$AAi?$AAs?$AAa?$AAb?$AAl?$AAe?$AA?3?$AA?5?$AAI?$AAn?$AAv?$AAa@ 00012ef8     oal_intr_mx25_topaz_v1:map.obj
 0001:00001f68       ??_C@_1DG@HOKLDENP@?$AA?$CL?$AAO?$AAE?$AAM?$AAI?$AAn?$AAt?$AAe?$AAr?$AAr?$AAu?$AAp?$AAt?$AAD?$AAi?$AAs?$AAa?$AAb?$AAl?$AAe?$AA?$CI?$AA?$CF?$AAd?$AA?$CJ?$AA?$AN?$AA?6?$AA?$AA@ 00012f68     oal_intr_mx25_topaz_v1:map.obj
 0001:00001fa0       ??_C@_1CI@OPHGDEL@?$AA?9?$AAO?$AAE?$AAM?$AAI?$AAn?$AAt?$AAe?$AAr?$AAr?$AAu?$AAp?$AAt?$AAM?$AAa?$AAs?$AAk?$AA?$AN?$AA?6?$AA?$AA@ 00012fa0     oal_intr_mx25_topaz_v1:map.obj
 0001:00001fc8       ??_C@_1GI@DLIDHGHH@?$AAE?$AAR?$AAR?$AAO?$AAR?$AA?3?$AA?5?$AAO?$AAE?$AAM?$AAI?$AAn?$AAt?$AAe?$AAr?$AAr?$AAu?$AAp?$AAt?$AAM?$AAa?$AAs?$AAk?$AA?3?$AA?5?$AAI?$AAn?$AAv?$AAa?$AAl?$AAi?$AAd@ 00012fc8     oal_intr_mx25_topaz_v1:map.obj
 0001:00002030       ??_C@_1DI@MFEEGIMP@?$AA?$CL?$AAO?$AAE?$AAM?$AAI?$AAn?$AAt?$AAe?$AAr?$AAr?$AAu?$AAp?$AAt?$AAM?$AAa?$AAs?$AAk?$AA?$CI?$AA?$CF?$AAd?$AA?0?$AA?5?$AA?$CF?$AAd?$AA?$CJ?$AA?$AN?$AA?6?$AA?$AA@ 00013030     oal_intr_mx25_topaz_v1:map.obj
 0001:00002068       ??_C@_1CI@IOEKFHHP@?$AA?9?$AAO?$AAE?$AAM?$AAI?$AAn?$AAt?$AAe?$AAr?$AAr?$AAu?$AAp?$AAt?$AAD?$AAo?$AAn?$AAe?$AA?$AN?$AA?6?$AA?$AA@ 00013068     oal_intr_mx25_topaz_v1:map.obj
 0001:00002090       ??_C@_1GI@FMDKDKKG@?$AAE?$AAR?$AAR?$AAO?$AAR?$AA?3?$AA?5?$AAO?$AAE?$AAM?$AAI?$AAn?$AAt?$AAe?$AAr?$AAr?$AAu?$AAp?$AAt?$AAD?$AAo?$AAn?$AAe?$AA?3?$AA?5?$AAI?$AAn?$AAv?$AAa?$AAl?$AAi?$AAd@ 00013090     oal_intr_mx25_topaz_v1:map.obj
 0001:000020f8       ??_C@_1DA@HAMHGFMF@?$AA?$CL?$AAO?$AAE?$AAM?$AAI?$AAn?$AAt?$AAe?$AAr?$AAr?$AAu?$AAp?$AAt?$AAD?$AAo?$AAn?$AAe?$AA?$CI?$AA?$CF?$AAd?$AA?$CJ?$AA?$AN?$AA?6?$AA?$AA@ 000130f8     oal_intr_mx25_topaz_v1:map.obj
 0001:000021b8       ??_C@_1DC@EGGJEANK@?$AA?9?$AAO?$AAE?$AAM?$AAI?$AAo?$AAC?$AAo?$AAn?$AAt?$AAr?$AAo?$AAl?$AA?$CI?$AAr?$AAc?$AA?5?$AA?$DN?$AA?5?$AA?$CF?$AAd?$AA?$CJ?$AA?$AN?$AA?6?$AA?$AA@ 000131b8     oal_ioctl_mx25_topaz_v1:ioctl.obj
 0001:000021f0       ??_C@_1HM@LHHDIECD@?$AAO?$AAE?$AAM?$AAI?$AAo?$AAC?$AAo?$AAn?$AAt?$AAr?$AAo?$AAl?$AA?3?$AA?5?$AAU?$AAn?$AAs?$AAu?$AAp?$AAp?$AAo?$AAr?$AAt?$AAe?$AAd?$AA?5?$AAC?$AAo?$AAd?$AAe?$AA?5?$AA0@ 000131f0     oal_ioctl_mx25_topaz_v1:ioctl.obj
 0001:00002270       ??_C@_1GA@KJDOLNLD@?$AA?$CL?$AAO?$AAE?$AAM?$AAI?$AAo?$AAC?$AAo?$AAn?$AAt?$AAr?$AAo?$AAl?$AA?$CI?$AA0?$AAx?$AA?$CF?$AAx?$AA?0?$AA?5?$AA0?$AAx?$AA?$CF?$AAx?$AA?0?$AA?5?$AA?$CF?$AAd?$AA?0?$AA?5?$AA0?$AAx@ 00013270     oal_ioctl_mx25_topaz_v1:ioctl.obj
 0001:00002360       ??_C@_1GK@FFHCMEEI@?$AAI?$AAN?$AAF?$AAO?$AA?3?$AA?5?$AAO?$AAE?$AAM?$AAP?$AAo?$AAw?$AAe?$AAr?$AAO?$AAf?$AAf?$AA?5?$AAl?$AAe?$AAa?$AAv?$AAi?$AAn?$AAg?$AA?5?$AAs?$AAu?$AAs?$AAp?$AAe?$AAn@ 00013360     oal_power_mx25_topaz_v1:off.obj
 0001:000023d0       ??_C@_1JG@FLHJIFLJ@?$AAI?$AAN?$AAF?$AAO?$AA?3?$AA?5?$AAO?$AAE?$AAM?$AAP?$AAo?$AAw?$AAe?$AAr?$AAO?$AAf?$AAf?$AA?5?$AAe?$AAn?$AAt?$AAe?$AAr?$AAi?$AAn?$AAg?$AA?5?$AAs?$AAu?$AAs?$AAp?$AAe@ 000133d0     oal_power_mx25_topaz_v1:off.obj
 0001:00002468       ??_C@_1HI@BGKFNECI@?$AAE?$AAR?$AAR?$AAO?$AAR?$AA?3?$AA?5?$AAO?$AAA?$AAL?$AAW?$AAa?$AAk?$AAe?$AAu?$AAp?$AAI?$AAn?$AAt?$AAe?$AAr?$AAr?$AAu?$AAp?$AAt?$AAE?$AAn?$AAa?$AAb?$AAl?$AAe?$AA?3@ 00013468     oal_power_mx25_topaz_v1:off.obj
 0001:00002570       ??_C@_1EE@EOJLKFMG@?$AA?$CL?$AAO?$AAA?$AAL?$AAI?$AAo?$AAC?$AAt?$AAl?$AAH?$AAa?$AAl?$AAE?$AAn?$AAa?$AAb?$AAl?$AAe?$AAW?$AAa?$AAk?$AAe?$AA?$CI?$AAr?$AAc?$AA?5?$AA?$DN?$AA?5?$AA?$CF?$AAd?$AA?$CJ?$AA?$AN@ 00013570     oal_power_mx25_topaz_v1:ioctl.obj
 0001:000025b4       ??_C@_1DO@BLFFHCCO@?$AAE?$AAR?$AAR?$AAO?$AAR?$AA?3?$AA?5?$AAO?$AAA?$AAL?$AAI?$AAo?$AAC?$AAt?$AAl?$AAH?$AAa?$AAl?$AAE?$AAn?$AAa?$AAb?$AAl?$AAe?$AAW?$AAa?$AAk?$AAe?$AA?3?$AA?5?$AA?$AA@ 000135b4     oal_power_mx25_topaz_v1:ioctl.obj
 0001:000025f4       ??_C@_1DG@KKNHDHOB@?$AAI?$AAn?$AAv?$AAa?$AAl?$AAi?$AAd?$AA?5?$AAS?$AAY?$AAS?$AAI?$AAN?$AAT?$AAR?$AA?5?$AAv?$AAa?$AAl?$AAu?$AAe?$AA?5?$AA?$CF?$AAd?$AA?$AN?$AA?6?$AA?$AA@ 000135f4     oal_power_mx25_topaz_v1:ioctl.obj
 0001:00002630       ??_C@_1EO@OMKOKHHJ@?$AA?$CL?$AAO?$AAA?$AAL?$AAI?$AAo?$AAC?$AAt?$AAl?$AAH?$AAa?$AAl?$AAE?$AAn?$AAa?$AAb?$AAl?$AAe?$AAW?$AAa?$AAk?$AAe?$AA?$CI?$AAs?$AAy?$AAs?$AAI?$AAn?$AAt?$AAr?$AA?5?$AA?$DN@ 00013630     oal_power_mx25_topaz_v1:ioctl.obj
 0001:00002680       ??_C@_1EG@KJIPIGDP@?$AA?$CL?$AAO?$AAA?$AAL?$AAI?$AAo?$AAC?$AAt?$AAl?$AAH?$AAa?$AAl?$AAD?$AAi?$AAs?$AAa?$AAb?$AAl?$AAe?$AAW?$AAa?$AAk?$AAe?$AA?$CI?$AAr?$AAc?$AA?5?$AA?$DN?$AA?5?$AA?$CF?$AAd?$AA?$CJ@ 00013680     oal_power_mx25_topaz_v1:ioctl.obj
 0001:000026c8       ??_C@_1EA@ENICBBFD@?$AAE?$AAR?$AAR?$AAO?$AAR?$AA?3?$AA?5?$AAO?$AAA?$AAL?$AAI?$AAo?$AAC?$AAt?$AAl?$AAH?$AAa?$AAl?$AAD?$AAi?$AAs?$AAa?$AAb?$AAl?$AAe?$AAW?$AAa?$AAk?$AAe?$AA?3?$AA?5?$AA?$AA@ 000136c8     oal_power_mx25_topaz_v1:ioctl.obj
 0001:00002708       ??_C@_1FA@IFHNBJAE@?$AA?$CL?$AAO?$AAA?$AAL?$AAI?$AAo?$AAC?$AAt?$AAl?$AAH?$AAa?$AAl?$AAD?$AAi?$AAs?$AAa?$AAb?$AAl?$AAe?$AAW?$AAa?$AAk?$AAe?$AA?$CI?$AAs?$AAy?$AAs?$AAI?$AAn?$AAt?$AAr?$AA?5@ 00013708     oal_power_mx25_topaz_v1:ioctl.obj
 0001:00002758       ??_C@_1GG@MBGEPMGD@?$AA?$CL?$AAO?$AAA?$AAL?$AAI?$AAo?$AAC?$AAt?$AAl?$AAH?$AAa?$AAl?$AAG?$AAe?$AAt?$AAW?$AAa?$AAk?$AAe?$AAS?$AAo?$AAu?$AAr?$AAc?$AAe?$AA?$CI?$AAr?$AAc?$AA?5?$AA?$DN?$AA?5?$AA?$CF@ 00013758     oal_power_mx25_topaz_v1:ioctl.obj
 0001:000027c0       ??_C@_1DI@DFOIFPDM@?$AA?$CL?$AAO?$AAA?$AAL?$AAI?$AAo?$AAC?$AAt?$AAl?$AAH?$AAa?$AAl?$AAG?$AAe?$AAt?$AAW?$AAa?$AAk?$AAe?$AAS?$AAo?$AAu?$AAr?$AAc?$AAe?$AA?$AN?$AA?6?$AA?$AA@ 000137c0     oal_power_mx25_topaz_v1:ioctl.obj
 0001:00002888       ??_C@_1DI@MKCLCMDC@?$AA?9?$AAO?$AAE?$AAM?$AAS?$AAe?$AAt?$AAA?$AAl?$AAa?$AAr?$AAm?$AAT?$AAi?$AAm?$AAe?$AA?$CI?$AAr?$AAc?$AA?5?$AA?$DN?$AA?5?$AA?$CF?$AAd?$AA?$CJ?$AA?$AN?$AA?6?$AA?$AA@ 00013888     oal_RTC_mx25_topaz_v1:alarm.obj
 0001:000028c0       ??_C@_1HC@CCDNFNOJ@?$AAE?$AAR?$AAR?$AAO?$AAR?$AA?3?$AA?5?$AAO?$AAE?$AAM?$AAS?$AAe?$AAt?$AAA?$AAl?$AAa?$AAr?$AAm?$AAT?$AAi?$AAm?$AAe?$AA?3?$AA?5?$AAN?$AAK?$AAS?$AAy?$AAs?$AAt?$AAe?$AAm@ 000138c0     oal_RTC_mx25_topaz_v1:alarm.obj
 0001:00002938       ??_C@_1GE@JGMJNPCG@?$AAE?$AAR?$AAR?$AAO?$AAR?$AA?3?$AA?5?$AAO?$AAE?$AAM?$AAS?$AAe?$AAt?$AAA?$AAl?$AAa?$AAr?$AAm?$AAT?$AAi?$AAm?$AAe?$AA?3?$AA?5?$AAU?$AAn?$AAs?$AAu?$AAp?$AAp?$AAo?$AAr@ 00013938     oal_RTC_mx25_topaz_v1:alarm.obj
 0001:000029a0       ??_C@_1FG@LDBAHALN@?$AA?$CL?$AAO?$AAE?$AAM?$AAS?$AAe?$AAt?$AAA?$AAl?$AAa?$AAr?$AAm?$AAT?$AAi?$AAm?$AAe?$AA?$CI?$AA?$CF?$AAd?$AA?1?$AA?$CF?$AAd?$AA?1?$AA?$CF?$AAd?$AA?5?$AA?$CF?$AAd?$AA?3?$AA?$CF?$AAd?$AA?3@ 000139a0     oal_RTC_mx25_topaz_v1:alarm.obj
 0001:00002a88       ??_C@_1GE@FHHIHPKE@?$AAE?$AAR?$AAR?$AAO?$AAR?$AA?3?$AA?5?$AAO?$AAA?$AAL?$AAR?$AAt?$AAc?$AAM?$AAa?$AAp?$AA?3?$AA?5?$AAR?$AAT?$AAC?$AA?5?$AAc?$AAr?$AAi?$AAt?$AAi?$AAc?$AAa?$AAl?$AA?5?$AAs@ 00013a88     oal_RTC_mx25_topaz_v1:rtc.obj
 0001:00002af0       ??_C@_1EO@PCFJJNAK@?$AAE?$AAR?$AAR?$AAO?$AAR?$AA?3?$AA?5?$AAO?$AAA?$AAL?$AAR?$AAt?$AAc?$AAM?$AAa?$AAp?$AA?3?$AA?5?$AAS?$AAR?$AAT?$AAC?$AA?5?$AAn?$AAu?$AAl?$AAl?$AA?5?$AAp?$AAo?$AAi?$AAn@ 00013af0     oal_RTC_mx25_topaz_v1:rtc.obj
 0001:00002b40       ??_C@_1EK@JDCHNJPO@?$AAR?$AAT?$AAC?$AA?5?$AAn?$AAo?$AAt?$AA?5?$AAr?$AAu?$AAn?$AAn?$AAi?$AAn?$AAg?$AA?4?$AA?5?$AAt?$AAu?$AAr?$AAn?$AAi?$AAn?$AAg?$AA?5?$AAi?$AAt?$AA?5?$AAo?$AAn?$AA?5?$AAn@ 00013b40     oal_RTC_mx25_topaz_v1:rtc.obj
 0001:00002b8c       ??_C@_1CM@FHGNKEPG@?$AAd?$AAr?$AAy?$AA?5?$AAi?$AAc?$AAe?$AA?5?$AAs?$AAt?$AAa?$AAt?$AAu?$AAs?$AA?5?$AA0?$AAx?$AA?$CF?$AAx?$AA?$AN?$AA?6?$AA?$AA@ 00013b8c     oal_RTC_mx25_topaz_v1:rtc.obj
 0001:00002bb8       ??_C@_1DM@INEGNAPC@?$AAd?$AAr?$AAy?$AA?5?$AAi?$AAc?$AAe?$AA?5?$AAi?$AAn?$AAi?$AAt?$AAi?$AAa?$AAl?$AA?5?$AAs?$AAt?$AAa?$AAt?$AAu?$AAs?$AA?5?$AA0?$AAx?$AA?$CF?$AAx?$AA?$AN?$AA?6?$AA?$AA@ 00013bb8     oal_RTC_mx25_topaz_v1:rtc.obj
 0001:00002bf4       ??_C@_1DO@FGGICPPB@?$AA?9?$AAO?$AAA?$AAL?$AAI?$AAo?$AAC?$AAt?$AAl?$AAH?$AAa?$AAl?$AAI?$AAn?$AAi?$AAt?$AAR?$AAT?$AAC?$AA?$CI?$AAr?$AAc?$AA?5?$AA?$DN?$AA?5?$AA?$CF?$AAd?$AA?$CJ?$AA?$AN?$AA?6?$AA?$AA@ 00013bf4     oal_RTC_mx25_topaz_v1:rtc.obj
 0001:00002c38       ??_C@_1FK@IDPOHODA@?$AAO?$AAA?$AAL?$AAI?$AAo?$AAC?$AAt?$AAl?$AAH?$AAa?$AAl?$AAI?$AAn?$AAi?$AAt?$AAR?$AAT?$AAC?$AA?$CI?$AA?$CF?$AAd?$AA?1?$AA?$CF?$AAd?$AA?1?$AA?$CF?$AAd?$AA?5?$AA?$CF?$AAd?$AA?3?$AA?$CF@ 00013c38     oal_RTC_mx25_topaz_v1:rtc.obj
 0001:00002c98       ??_C@_1FO@ODJLIDFO@?$AAE?$AAR?$AAR?$AAO?$AAR?$AA?3?$AA?5?$AAO?$AAA?$AAL?$AAI?$AAo?$AAC?$AAt?$AAl?$AAH?$AAa?$AAl?$AAI?$AAn?$AAi?$AAt?$AAR?$AAT?$AAC?$AA?3?$AA?5?$AAI?$AAn?$AAv?$AAa?$AAl@ 00013c98     oal_RTC_mx25_topaz_v1:rtc.obj
 0001:00002cf8       ??_C@_1DG@PECFOPGF@?$AA?$CL?$AAO?$AAA?$AAL?$AAI?$AAo?$AAC?$AAt?$AAl?$AAH?$AAa?$AAl?$AAI?$AAn?$AAi?$AAt?$AAR?$AAT?$AAC?$AA?$CI?$AA?4?$AA?4?$AA?4?$AA?$CJ?$AA?$AN?$AA?6?$AA?$AA@ 00013cf8     oal_RTC_mx25_topaz_v1:rtc.obj
 0001:00002d30       ??_C@_1GG@MNNCNIB@?$AA?9?$AAO?$AAE?$AAM?$AAG?$AAe?$AAt?$AAR?$AAe?$AAa?$AAl?$AAT?$AAi?$AAm?$AAe?$AA?$CI?$AAr?$AAc?$AA?5?$AA?$DN?$AA?5?$AA?$CF?$AAd?$AA?0?$AA?5?$AA?$CF?$AAd?$AA?1?$AA?$CF?$AAd?$AA?1?$AA?$CF@ 00013d30     oal_RTC_mx25_topaz_v1:rtc.obj
 0001:00002d98       ??_C@_1FG@FLJPFOHI@?$AAE?$AAR?$AAR?$AAO?$AAR?$AA?3?$AA?5?$AAO?$AAE?$AAM?$AAG?$AAe?$AAt?$AAR?$AAe?$AAa?$AAl?$AAT?$AAi?$AAm?$AAe?$AA?3?$AA?5?$AAO?$AAA?$AAL?$AAR?$AAt?$AAc?$AAM?$AAa?$AAp@ 00013d98     oal_RTC_mx25_topaz_v1:rtc.obj
 0001:00002df0       ??_C@_1CE@MMIOOJN@?$AA?$CL?$AAO?$AAE?$AAM?$AAG?$AAe?$AAt?$AAR?$AAe?$AAa?$AAl?$AAT?$AAi?$AAm?$AAe?$AA?$AN?$AA?6?$AA?$AA@ 00013df0     oal_RTC_mx25_topaz_v1:rtc.obj
 0001:00002e14       ??_C@_1DG@MOFFCBMN@?$AA?9?$AAO?$AAE?$AAM?$AAS?$AAe?$AAt?$AAR?$AAe?$AAa?$AAl?$AAT?$AAi?$AAm?$AAe?$AA?$CI?$AAr?$AAc?$AA?5?$AA?$DN?$AA?5?$AA?$CF?$AAd?$AA?$CJ?$AA?$AN?$AA?6?$AA?$AA@ 00013e14     oal_RTC_mx25_topaz_v1:rtc.obj
 0001:00002e50       ??_C@_1HA@FDHJPCFE@?$AAE?$AAR?$AAR?$AAO?$AAR?$AA?3?$AA?5?$AAO?$AAE?$AAM?$AAS?$AAe?$AAt?$AAR?$AAe?$AAa?$AAl?$AAT?$AAi?$AAm?$AAe?$AA?3?$AA?5?$AAN?$AAK?$AAS?$AAy?$AAs?$AAt?$AAe?$AAm?$AAT@ 00013e50     oal_RTC_mx25_topaz_v1:rtc.obj
 0001:00002ec0       ??_C@_1GC@DPKGAKNF@?$AAE?$AAR?$AAR?$AAO?$AAR?$AA?3?$AA?5?$AAO?$AAE?$AAM?$AAS?$AAe?$AAt?$AAR?$AAe?$AAa?$AAl?$AAT?$AAi?$AAm?$AAe?$AA?3?$AA?5?$AAU?$AAn?$AAs?$AAu?$AAp?$AAp?$AAo?$AAr?$AAt@ 00013ec0     oal_RTC_mx25_topaz_v1:rtc.obj
 0001:00002f28       ??_C@_1FG@OCPECIDD@?$AAE?$AAR?$AAR?$AAO?$AAR?$AA?3?$AA?5?$AAO?$AAE?$AAM?$AAS?$AAe?$AAt?$AAR?$AAe?$AAa?$AAl?$AAT?$AAi?$AAm?$AAe?$AA?3?$AA?5?$AAO?$AAA?$AAL?$AAR?$AAt?$AAc?$AAM?$AAa?$AAp@ 00013f28     oal_RTC_mx25_topaz_v1:rtc.obj
 0001:00002f80       ??_C@_1FE@NLGIDKMA@?$AA?$CL?$AAO?$AAE?$AAM?$AAS?$AAe?$AAt?$AAR?$AAe?$AAa?$AAl?$AAT?$AAi?$AAm?$AAe?$AA?$CI?$AA?$CF?$AAd?$AA?1?$AA?$CF?$AAd?$AA?1?$AA?$CF?$AAd?$AA?5?$AA?$CF?$AAd?$AA?3?$AA?$CF?$AAd?$AA?3?$AA?$CF@ 00013f80     oal_RTC_mx25_topaz_v1:rtc.obj
 0001:00002fd4       ??_C@_1DE@DAHNLBLJ@?$AA?9?$AAO?$AAA?$AAL?$AAP?$AAA?$AAt?$AAo?$AAV?$AAA?$AA?$CI?$AAv?$AAa?$AA?5?$AA?$DN?$AA?5?$AA0?$AAx?$AA?$CF?$AA0?$AA8?$AAx?$AA?$CJ?$AA?$AN?$AA?6?$AA?$AA@ 00013fd4     oal_memory_arm:memory.obj
 0001:00003008       ??_C@_1CO@JEIJEAKF@?$AA?$CL?$AAO?$AAA?$AAL?$AAP?$AAA?$AAt?$AAo?$AAV?$AAA?$AA?$CI?$AA0?$AAx?$AA?$CF?$AAx?$AA?0?$AA?5?$AA?$CF?$AAd?$AA?$CJ?$AA?$AN?$AA?6?$AA?$AA@ 00014008     oal_memory_arm:memory.obj
 0001:00003038       ??_C@_1DA@BBOHBBNH@?$AA?9?$AAO?$AAA?$AAL?$AAV?$AAA?$AAt?$AAo?$AAP?$AAA?$AA?$CI?$AAp?$AAa?$AA?5?$AA?$DN?$AA?5?$AA0?$AAx?$AA?$CF?$AAx?$AA?$CJ?$AA?$AN?$AA?6?$AA?$AA@ 00014038     oal_memory_arm:memory.obj
 0001:00003068       ??_C@_1CK@LKNIEAFP@?$AA?$CL?$AAO?$AAA?$AAL?$AAV?$AAA?$AAt?$AAo?$AAP?$AAA?$AA?$CI?$AA0?$AAx?$AA?$CF?$AA0?$AA8?$AAx?$AA?$CJ?$AA?$AN?$AA?6?$AA?$AA@ 00014068     oal_memory_arm:memory.obj
 0001:00003128       ??_C@_1DC@ONFHCFK@?$AA?9?$AAO?$AAE?$AAM?$AAP?$AAr?$AAo?$AAf?$AAi?$AAl?$AAe?$AAT?$AAi?$AAm?$AAe?$AAr?$AAE?$AAn?$AAa?$AAb?$AAl?$AAe?$AA?$AN?$AA?6?$AA?$AA@ 00014128     oal_profiler_gpt_mx25_topaz_v1:profiler.obj
 0001:00003160       ??_C@_1FG@KKJMBHIF@?$AAO?$AAE?$AAM?$AAP?$AAr?$AAo?$AAf?$AAi?$AAl?$AAe?$AAT?$AAi?$AAm?$AAe?$AAr?$AAE?$AAn?$AAa?$AAb?$AAl?$AAe?$AA?3?$AA?5?$AAc?$AAo?$AAu?$AAn?$AAt?$AAs?$AAP?$AAe?$AAr@ 00014160     oal_profiler_gpt_mx25_topaz_v1:profiler.obj
 0001:000031b8       ??_C@_1DK@OJEFEGCL@?$AA?$CL?$AAO?$AAE?$AAM?$AAP?$AAr?$AAo?$AAf?$AAi?$AAl?$AAe?$AAT?$AAi?$AAm?$AAe?$AAr?$AAE?$AAn?$AAa?$AAb?$AAl?$AAe?$AA?$CI?$AA?$CF?$AAd?$AA?$CJ?$AA?$AN?$AA?6?$AA?$AA@ 000141b8     oal_profiler_gpt_mx25_topaz_v1:profiler.obj
 0001:000031f4       ??_C@_1DE@DGCDHBJ@?$AA?9?$AAO?$AAE?$AAM?$AAP?$AAr?$AAo?$AAf?$AAi?$AAl?$AAe?$AAT?$AAi?$AAm?$AAe?$AAr?$AAD?$AAi?$AAs?$AAa?$AAb?$AAl?$AAe?$AA?$AN?$AA?6?$AA?$AA@ 000141f4     oal_profiler_gpt_mx25_topaz_v1:profiler.obj
 0001:00003228       ??_C@_1DI@ICCHIFPG@?$AA?$CL?$AAO?$AAE?$AAM?$AAP?$AAr?$AAo?$AAf?$AAi?$AAl?$AAe?$AAT?$AAi?$AAm?$AAe?$AAr?$AAD?$AAi?$AAs?$AAa?$AAb?$AAl?$AAe?$AA?$CI?$AA?$CJ?$AA?$AN?$AA?6?$AA?$AA@ 00014228     oal_profiler_gpt_mx25_topaz_v1:profiler.obj
 0001:000032f0       ??_C@_1GM@LBPDAPNJ@?$AAI?$AAN?$AAF?$AAO?$AA?3?$AAO?$AAA?$AAL?$AAL?$AAo?$AAg?$AAS?$AAe?$AAt?$AAZ?$AAo?$AAn?$AAe?$AAs?$AA?3?$AA?5?$AAd?$AAp?$AAC?$AAu?$AAr?$AAS?$AAe?$AAt?$AAt?$AAi?$AAn@ 000142f0     oal_log:debug.obj
 0001:00003418       ??_C@_1KC@KHIEGOFB@?$AAO?$AAA?$AAL?$AAI?$AAs?$AAP?$AAr?$AAo?$AAc?$AAe?$AAs?$AAs?$AAo?$AAr?$AAF?$AAe?$AAa?$AAt?$AAu?$AAr?$AAe?$AAP?$AAr?$AAe?$AAs?$AAe?$AAn?$AAt?$AA?3?$AA?5?$AAI?$AAD@ 00014418     oal_misc_arm:feature.obj
 0001:000035e0       ??_C@_1DM@OCLJLKJN@?$AA?5?$AA?5?$AA?5?$AA?5?$AAP?$AAe?$AAr?$AAi?$AAp?$AAh?$AA?5?$AAC?$AAl?$AAk?$AA?5?$AAU?$AAA?$AAR?$AAT?$AA?5?$AA?$DN?$AA?5?$AA?$CF?$AAd?$AA?5?$AAH?$AAz?$AA?$AN?$AA?6?$AA?$AA@ 000145e0     bspcmn:bspargs.obj
 0001:0000361c       ??_C@_1DM@BGNEBGOE@?$AA?5?$AA?5?$AA?5?$AA?5?$AAP?$AAe?$AAr?$AAi?$AAp?$AAh?$AA?5?$AAC?$AAl?$AAk?$AA?5?$AAS?$AAS?$AAI?$AA2?$AA?5?$AA?$DN?$AA?5?$AA?$CF?$AAd?$AA?5?$AAH?$AAz?$AA?$AN?$AA?6?$AA?$AA@ 0001461c     bspcmn:bspargs.obj
 0001:00003658       ??_C@_1DM@EOMKLPMM@?$AA?5?$AA?5?$AA?5?$AA?5?$AAP?$AAe?$AAr?$AAi?$AAp?$AAh?$AA?5?$AAC?$AAl?$AAk?$AA?5?$AAS?$AAS?$AAI?$AA1?$AA?5?$AA?$DN?$AA?5?$AA?$CF?$AAd?$AA?5?$AAH?$AAz?$AA?$AN?$AA?6?$AA?$AA@ 00014658     bspcmn:bspargs.obj
 0001:00003694       ??_C@_1DM@CJNLEDDI@?$AA?5?$AA?5?$AA?5?$AA?5?$AAP?$AAe?$AAr?$AAi?$AAp?$AAh?$AA?5?$AAC?$AAl?$AAk?$AA?5?$AAS?$AAI?$AAM?$AA2?$AA?5?$AA?$DN?$AA?5?$AA?$CF?$AAd?$AA?5?$AAH?$AAz?$AA?$AN?$AA?6?$AA?$AA@ 00014694     bspcmn:bspargs.obj
 0001:000036d0       ??_C@_1DM@HBMFOKBA@?$AA?5?$AA?5?$AA?5?$AA?5?$AAP?$AAe?$AAr?$AAi?$AAp?$AAh?$AA?5?$AAC?$AAl?$AAk?$AA?5?$AAS?$AAI?$AAM?$AA1?$AA?5?$AA?$DN?$AA?5?$AA?$CF?$AAd?$AA?5?$AAH?$AAz?$AA?$AN?$AA?6?$AA?$AA@ 000146d0     bspcmn:bspargs.obj
 0001:0000370c       ??_C@_1DK@MIDNNIPL@?$AA?5?$AA?5?$AA?5?$AA?5?$AAP?$AAe?$AAr?$AAi?$AAp?$AAh?$AA?5?$AAC?$AAl?$AAk?$AA?5?$AAP?$AAW?$AAM?$AA?5?$AA?$DN?$AA?5?$AA?$CF?$AAd?$AA?5?$AAH?$AAz?$AA?$AN?$AA?6?$AA?$AA@ 0001470c     bspcmn:bspargs.obj
 0001:00003748       ??_C@_1DO@GMICDJDG@?$AA?5?$AA?5?$AA?5?$AA?5?$AAP?$AAe?$AAr?$AAi?$AAp?$AAh?$AA?5?$AAC?$AAl?$AAk?$AA?5?$AAO?$AAW?$AAI?$AAR?$AAE?$AA?5?$AA?$DN?$AA?5?$AA?$CF?$AAd?$AA?5?$AAH?$AAz?$AA?$AN?$AA?6?$AA?$AA@ 00014748     bspcmn:bspargs.obj
 0001:00003788       ??_C@_1DK@PEAOHMIM@?$AA?5?$AA?5?$AA?5?$AA?5?$AAP?$AAe?$AAr?$AAi?$AAp?$AAh?$AA?5?$AAC?$AAl?$AAk?$AA?5?$AAN?$AAF?$AAC?$AA?5?$AA?$DN?$AA?5?$AA?$CF?$AAd?$AA?5?$AAH?$AAz?$AA?$AN?$AA?6?$AA?$AA@ 00014788     bspcmn:bspargs.obj
 0001:000037c4       ??_C@_1DM@EONHEPCP@?$AA?5?$AA?5?$AA?5?$AA?5?$AAP?$AAe?$AAr?$AAi?$AAp?$AAh?$AA?5?$AAC?$AAl?$AAk?$AA?5?$AAL?$AAC?$AAD?$AAC?$AA?5?$AA?$DN?$AA?5?$AA?$CF?$AAd?$AA?5?$AAH?$AAz?$AA?$AN?$AA?6?$AA?$AA@ 000147c4     bspcmn:bspargs.obj
 0001:00003800       ??_C@_1DK@DLMOJFOL@?$AA?5?$AA?5?$AA?5?$AA?5?$AAP?$AAe?$AAr?$AAi?$AAp?$AAh?$AA?5?$AAC?$AAl?$AAk?$AA?5?$AAI?$AA2?$AAC?$AA?5?$AA?$DN?$AA?5?$AA?$CF?$AAd?$AA?5?$AAH?$AAz?$AA?$AN?$AA?6?$AA?$AA@ 00014800     bspcmn:bspargs.obj
 0001:0000383c       ??_C@_1DK@CDOLKHPK@?$AA?5?$AA?5?$AA?5?$AA?5?$AAP?$AAe?$AAr?$AAi?$AAp?$AAh?$AA?5?$AAC?$AAl?$AAk?$AA?5?$AAG?$AAP?$AAT?$AA?5?$AA?$DN?$AA?5?$AA?$CF?$AAd?$AA?5?$AAH?$AAz?$AA?$AN?$AA?6?$AA?$AA@ 0001483c     bspcmn:bspargs.obj
 0001:00003878       ??_C@_1EA@MPFCNGCJ@?$AA?5?$AA?5?$AA?5?$AA?5?$AAP?$AAe?$AAr?$AAi?$AAp?$AAh?$AA?5?$AAC?$AAl?$AAk?$AA?5?$AAE?$AAS?$AAD?$AAH?$AAC?$AA2?$AA?5?$AA?$DN?$AA?5?$AA?$CF?$AAd?$AA?5?$AAH?$AAz?$AA?$AN?$AA?6?$AA?$AA@ 00014878     bspcmn:bspargs.obj
 0001:000038b8       ??_C@_1EA@JHEMHPAB@?$AA?5?$AA?5?$AA?5?$AA?5?$AAP?$AAe?$AAr?$AAi?$AAp?$AAh?$AA?5?$AAC?$AAl?$AAk?$AA?5?$AAE?$AAS?$AAD?$AAH?$AAC?$AA1?$AA?5?$AA?$DN?$AA?5?$AA?$CF?$AAd?$AA?5?$AAH?$AAz?$AA?$AN?$AA?6?$AA?$AA@ 000148b8     bspcmn:bspargs.obj
 0001:000038f8       ??_C@_1DM@JHCBKDAO@?$AA?5?$AA?5?$AA?5?$AA?5?$AAP?$AAe?$AAr?$AAi?$AAp?$AAh?$AA?5?$AAC?$AAl?$AAk?$AA?5?$AAE?$AAS?$AAA?$AAI?$AA?5?$AA?$DN?$AA?5?$AA?$CF?$AAd?$AA?5?$AAH?$AAz?$AA?$AN?$AA?6?$AA?$AA@ 000148f8     bspcmn:bspargs.obj
 0001:00003934       ??_C@_1DM@IFJDDBGO@?$AA?5?$AA?5?$AA?5?$AA?5?$AAP?$AAe?$AAr?$AAi?$AAp?$AAh?$AA?5?$AAC?$AAl?$AAk?$AA?5?$AAE?$AAP?$AAI?$AAT?$AA?5?$AA?$DN?$AA?5?$AA?$CF?$AAd?$AA?5?$AAH?$AAz?$AA?$AN?$AA?6?$AA?$AA@ 00014934     bspcmn:bspargs.obj
 0001:00003970       ??_C@_1DK@JCCOAGIN@?$AA?5?$AA?5?$AA?5?$AA?5?$AAP?$AAe?$AAr?$AAi?$AAp?$AAh?$AA?5?$AAC?$AAl?$AAk?$AA?5?$AAC?$AAS?$AAI?$AA?5?$AA?$DN?$AA?5?$AA?$CF?$AAd?$AA?5?$AAH?$AAz?$AA?$AN?$AA?6?$AA?$AA@ 00014970     bspcmn:bspargs.obj
 0001:000039ac       ??_C@_1DA@OBKCEEDF@?$AA?5?$AA?5?$AA?5?$AA?5?$AAU?$AAS?$AAB?$AA?5?$AAC?$AAL?$AAO?$AAC?$AAK?$AA?5?$AA?$DN?$AA?5?$AA?$CF?$AAd?$AA?5?$AAH?$AAz?$AA?$AN?$AA?6?$AA?$AA@ 000149ac     bspcmn:bspargs.obj
 0001:000039dc       ??_C@_1DC@HLPKBKNH@?$AA?5?$AA?5?$AA?5?$AA?5?$AAI?$AAP?$AAG?$AA?5?$AAC?$AAL?$AAO?$AAC?$AAK?$AA?5?$AA?5?$AA?$DN?$AA?5?$AA?$CF?$AAd?$AA?5?$AAH?$AAz?$AA?$AN?$AA?6?$AA?$AA@ 000149dc     bspcmn:bspargs.obj
 0001:00003a10       ??_C@_1DC@CKMNKMMI@?$AA?5?$AA?5?$AA?5?$AA?5?$AAA?$AAH?$AAB?$AA?5?$AAC?$AAL?$AAO?$AAC?$AAK?$AA?5?$AA?5?$AA?$DN?$AA?5?$AA?$CF?$AAd?$AA?5?$AAH?$AAz?$AA?$AN?$AA?6?$AA?$AA@ 00014a10     bspcmn:bspargs.obj
 0001:00003a44       ??_C@_1DC@IAJIALLM@?$AA?5?$AA?5?$AA?5?$AA?5?$AAA?$AAR?$AAM?$AA?5?$AAC?$AAL?$AAO?$AAC?$AAK?$AA?5?$AA?5?$AA?$DN?$AA?5?$AA?$CF?$AAd?$AA?5?$AAH?$AAz?$AA?$AN?$AA?6?$AA?$AA@ 00014a44     bspcmn:bspargs.obj
 0001:00003a78       ??_C@_1CO@IOOCOMMB@?$AA?5?$AA?5?$AA?5?$AA?5?$AAU?$AAS?$AAB?$AA?5?$AAP?$AAL?$AAL?$AA?5?$AA?5?$AA?$DN?$AA?5?$AA?$CF?$AAd?$AA?5?$AAH?$AAz?$AA?$AN?$AA?6?$AA?$AA@ 00014a78     bspcmn:bspargs.obj
 0001:00003aa8       ??_C@_1CO@LHEJCJEH@?$AA?5?$AA?5?$AA?5?$AA?5?$AAM?$AAC?$AAU?$AA?5?$AAP?$AAL?$AAL?$AA?5?$AA?5?$AA?$DN?$AA?5?$AA?$CF?$AAd?$AA?5?$AAH?$AAz?$AA?$AN?$AA?6?$AA?$AA@ 00014aa8     bspcmn:bspargs.obj
 0001:00003ad8       ??_C@_1DG@IJHKIPGD@?$AAB?$AAS?$AAP?$AA?5?$AAC?$AAl?$AAo?$AAc?$AAk?$AA?5?$AAC?$AAo?$AAn?$AAf?$AAi?$AAg?$AAu?$AAr?$AAa?$AAt?$AAi?$AAo?$AAn?$AA?3?$AA?$AN?$AA?6?$AA?$AA@ 00014ad8     bspcmn:bspargs.obj
 0001:00003ba0       ??_C@_1FE@FFNPEPPH@?$AAH?$AAa?$AAr?$AAd?$AAw?$AAa?$AAr?$AAe?$AA?5?$AAf?$AAl?$AAo?$AAw?$AA?5?$AAc?$AAo?$AAn?$AAt?$AAr?$AAo?$AAl?$AA?5?$AAi?$AAs?$AA?5?$AAn?$AAo?$AAt?$AA?5?$AAs?$AAu?$AAp@ 00014ba0     serialutils:serialutils.obj
 0001:00003bf8       ??_C@_1KG@BFMCBNEC@?$AAC?$AA?3?$AA?2?$AAW?$AAI?$AAN?$AAC?$AAE?$AAR?$AAO?$AAO?$AAT?$AAS?$AA?2?$AAT?$AAo?$AAp?$AAa?$AAz?$AA?2?$AAW?$AAI?$AAN?$AAC?$AAE?$AA6?$AA0?$AA0?$AA?2?$AAP?$AAL?$AAA@ 00014bf8     serialutils:serialutils.obj
 0001:00003d30       ??_C@_1EA@DJGHLELP@?$AA?9?$AAO?$AAA?$AAL?$AAA?$AAr?$AAg?$AAs?$AAQ?$AAu?$AAe?$AAr?$AAy?$AA?$CI?$AAp?$AAD?$AAa?$AAt?$AAa?$AA?5?$AA?$DN?$AA?5?$AA0?$AAx?$AA?$CF?$AA0?$AA8?$AAx?$AA?$CJ?$AA?$AN?$AA?6?$AA?$AA@ 00014d30     args:args.obj
 0001:00003d70       ??_C@_1CI@CLMEBIJE@?$AA?$CL?$AAO?$AAA?$AAL?$AAA?$AAr?$AAg?$AAs?$AAQ?$AAu?$AAe?$AAr?$AAy?$AA?$CI?$AA?$CF?$AAd?$AA?$CJ?$AA?$AN?$AA?6?$AA?$AA@ 00014d70     args:args.obj
 0001:00003e28       ??_C@_1DC@HNHAGOEA@?$AA?5?$AAR?$AAe?$AAg?$AAu?$AAl?$AAa?$AAt?$AAo?$AAr?$AA?5?$AAn?$AAo?$AAt?$AA?5?$AAs?$AAu?$AAp?$AAp?$AAo?$AAr?$AAt?$AAe?$AAd?$AA?$AA@ 00014e28     pmicutils:mc34704utils.obj
 0001:00003e60       ??_C@_1EO@LPFNDCLA@?$AAR?$AAe?$AAg?$AAu?$AAl?$AAa?$AAt?$AAo?$AAr?$AA?5?$AA8?$AA?5?$AAm?$AAa?$AAn?$AAa?$AAg?$AAe?$AAm?$AAe?$AAn?$AAt?$AA?5?$AAn?$AAo?$AAt?$AA?5?$AAi?$AAm?$AAp?$AAl?$AAe@ 00014e60     pmicutils:mc34704utils.obj
 0001:00003eb0       ??_C@_1EO@KLNCGMFD@?$AAR?$AAe?$AAg?$AAu?$AAl?$AAa?$AAt?$AAo?$AAr?$AA?5?$AA7?$AA?5?$AAm?$AAa?$AAn?$AAa?$AAg?$AAe?$AAm?$AAe?$AAn?$AAt?$AA?5?$AAn?$AAo?$AAt?$AA?5?$AAi?$AAm?$AAp?$AAl?$AAe@ 00014eb0     pmicutils:mc34704utils.obj
 0001:00003f00       ??_C@_1EO@OBBFGDMA@?$AAR?$AAe?$AAg?$AAu?$AAl?$AAa?$AAt?$AAo?$AAr?$AA?5?$AA6?$AA?5?$AAm?$AAa?$AAn?$AAa?$AAg?$AAe?$AAm?$AAe?$AAn?$AAt?$AA?5?$AAn?$AAo?$AAt?$AA?5?$AAi?$AAm?$AAp?$AAl?$AAe@ 00014f00     pmicutils:mc34704utils.obj
 0001:00003f50       ??_C@_1EO@DOFMHDHF@?$AAR?$AAe?$AAg?$AAu?$AAl?$AAa?$AAt?$AAo?$AAr?$AA?5?$AA5?$AA?5?$AAm?$AAa?$AAn?$AAa?$AAg?$AAe?$AAm?$AAe?$AAn?$AAt?$AA?5?$AAn?$AAo?$AAt?$AA?5?$AAi?$AAm?$AAp?$AAl?$AAe@ 00014f50     pmicutils:mc34704utils.obj
 0001:00003fa0       ??_C@_1EO@HEJLHMOG@?$AAR?$AAe?$AAg?$AAu?$AAl?$AAa?$AAt?$AAo?$AAr?$AA?5?$AA4?$AA?5?$AAm?$AAa?$AAn?$AAa?$AAg?$AAe?$AAm?$AAe?$AAn?$AAt?$AA?5?$AAn?$AAo?$AAt?$AA?5?$AAi?$AAm?$AAp?$AAl?$AAe@ 00014fa0     pmicutils:mc34704utils.obj
 0001:00003ff0       ??_C@_1EO@MODBELHI@?$AAR?$AAe?$AAg?$AAu?$AAl?$AAa?$AAt?$AAo?$AAr?$AA?5?$AA1?$AA?5?$AAm?$AAa?$AAn?$AAa?$AAg?$AAe?$AAm?$AAe?$AAn?$AAt?$AA?5?$AAn?$AAo?$AAt?$AA?5?$AAi?$AAm?$AAp?$AAl?$AAe@ 00014ff0     pmicutils:mc34704utils.obj
 0001:00004040       ??_C@_1CA@EIFFEMAD@?$AAN?$AAo?$AAt?$AA?5?$AAi?$AAm?$AAp?$AAl?$AAe?$AAm?$AAe?$AAn?$AAt?$AAe?$AAd?$AA?$AA@ 00015040     pmicutils:mc34704utils.obj
 0001:00004060       ??_C@_1GI@CBHCCGLJ@?$AAP?$AAm?$AAi?$AAc?$AAG?$AAe?$AAt?$AAR?$AAe?$AAg?$AAi?$AAs?$AAt?$AAe?$AAr?$AA?3?$AA?5?$AAO?$AAA?$AAL?$AAI?$AA2?$AAc?$AAR?$AAe?$AAa?$AAd?$AAD?$AAa?$AAt?$AAa?$AA?5@ 00015060     pmicutils:mc34704utils.obj
 0001:000040c8       ??_C@_1GE@FGMCNOJB@?$AAP?$AAm?$AAi?$AAc?$AAG?$AAe?$AAt?$AAR?$AAe?$AAg?$AAi?$AAs?$AAt?$AAe?$AAr?$AA?3?$AA?5?$AAO?$AAA?$AAL?$AAI?$AA2?$AAc?$AAW?$AAr?$AAi?$AAt?$AAe?$AAD?$AAa?$AAt?$AAa@ 000150c8     pmicutils:mc34704utils.obj
 0001:00004130       ??_C@_1FM@GFAOPLEL@?$AAP?$AAm?$AAi?$AAc?$AAG?$AAe?$AAt?$AAR?$AAe?$AAg?$AAi?$AAs?$AAt?$AAe?$AAr?$AA?3?$AA?5?$AAO?$AAA?$AAL?$AAI?$AA2?$AAc?$AAG?$AAe?$AAn?$AAe?$AAr?$AAa?$AAt?$AAe?$AAS@ 00015130     pmicutils:mc34704utils.obj
 0001:000042a0       ??_C@_1EO@BIINPADA@?$AAO?$AAA?$AAL?$AAP?$AAm?$AAi?$AAc?$AAI?$AAn?$AAi?$AAt?$AA?3?$AA?5?$AAO?$AAA?$AAL?$AAP?$AAA?$AAt?$AAo?$AAU?$AAA?$AA?5?$AAr?$AAe?$AAt?$AAu?$AAr?$AAn?$AAe?$AAd?$AA?5@ 000152a0     i2cutils:i2cutils.obj
 0001:000042f0       ??_C@_1EK@BGCNBCKF@?$AAO?$AAA?$AAL?$AAI?$AA2?$AAc?$AAI?$AAn?$AAi?$AAt?$AA?3?$AA?5?$AAI?$AAO?$AAM?$AAU?$AAX?$AAC?$AA?5?$AAm?$AAa?$AAp?$AAp?$AAi?$AAn?$AAg?$AA?5?$AAf?$AAa?$AAi?$AAl?$AAe@ 000152f0     i2cutils:i2cutils.obj
 0001:00004340       ??_C@_1FG@HMBKJBKF@?$AAO?$AAA?$AAL?$AAI?$AA2?$AAc?$AAI?$AAn?$AAi?$AAt?$AA?3?$AA?5?$AAT?$AAr?$AAy?$AAi?$AAn?$AAg?$AA?5?$AAt?$AAo?$AA?5?$AAi?$AAn?$AAi?$AAt?$AA?5?$AAI?$AA2?$AAC?$AA?5?$AAI@ 00015340     i2cutils:i2cutils.obj
 0001:00004398       ??_C@_1DK@MPINBAIN@?$AA?$CF?$AAs?$AA?3?$AA?5?$AAB?$AAu?$AAs?$AA?5?$AAb?$AAu?$AAs?$AAy?$AA?5?$AAf?$AAo?$AAr?$AA?5?$AA?$CF?$AAd?$AA?5?$AAc?$AAy?$AAc?$AAl?$AAe?$AAs?$AA?$AN?$AA?6?$AA?$AA@ 00015398     i2cutils:i2cutils.obj
 0001:000043d4       ??_C@_1CI@JNEOMLK@?$AAO?$AAA?$AAL?$AAI?$AA2?$AAc?$AAG?$AAe?$AAn?$AAe?$AAr?$AAa?$AAt?$AAe?$AAS?$AAt?$AAa?$AAr?$AAt?$AA?$AA@ 000153d4     i2cutils:i2cutils.obj
 0001:00004400       ??_C@_1EI@LDHHPPEC@?$AA?$CF?$AAs?$AA?3?$AA?5?$AAB?$AAu?$AAs?$AA?5?$AAn?$AAo?$AAt?$AA?5?$AAc?$AAl?$AAe?$AAa?$AAr?$AAe?$AAd?$AA?5?$AAf?$AAo?$AAr?$AA?5?$AA?$CF?$AAd?$AA?5?$AAc?$AAy?$AAc?$AAl?$AAe@ 00015400     i2cutils:i2cutils.obj
 0001:00004448       ??_C@_1CG@KGNMMGFF@?$AAO?$AAA?$AAL?$AAI?$AA2?$AAc?$AAG?$AAe?$AAn?$AAe?$AAr?$AAa?$AAt?$AAe?$AAS?$AAt?$AAo?$AAp?$AA?$AA@ 00015448     i2cutils:i2cutils.obj
 0001:00004470       ??_C@_1CM@BMDDLKDO@?$AA?9?$AAO?$AAE?$AAM?$AAC?$AAa?$AAc?$AAh?$AAe?$AAR?$AAa?$AAn?$AAg?$AAe?$AAF?$AAl?$AAu?$AAs?$AAh?$AA?$AN?$AA?6?$AA?$AA@ 00015470     oal_cache_arm926:flush.obj
 0001:000044a0       ??_C@_1FE@FFFKHHBK@?$AA?$CL?$AAO?$AAE?$AAM?$AAC?$AAa?$AAc?$AAh?$AAe?$AAR?$AAa?$AAn?$AAg?$AAe?$AAF?$AAl?$AAu?$AAs?$AAh?$AA?$CI?$AA0?$AAx?$AA?$CF?$AA0?$AA8?$AAx?$AA?0?$AA?5?$AA?$CF?$AAd?$AA?0?$AA?5@ 000154a0     oal_cache_arm926:flush.obj
 0001:00004588       ??_C@_1DM@POOLLMMJ@?$AA?9?$AAB?$AAS?$AAP?$AAI?$AAn?$AAt?$AAr?$AAR?$AAe?$AAq?$AAu?$AAe?$AAs?$AAt?$AAI?$AAr?$AAq?$AA?$CI?$AAr?$AAc?$AA?5?$AA?$DN?$AA?5?$AA?$CF?$AAd?$AA?$CJ?$AA?$AN?$AA?6?$AA?$AA@ 00015588     oal:intr.obj
 0001:000045c8       ??_C@_1HM@BJHIHKHI@?$AA?$CL?$AAB?$AAS?$AAP?$AAI?$AAn?$AAt?$AAr?$AAR?$AAe?$AAq?$AAu?$AAe?$AAs?$AAt?$AAI?$AAr?$AAq?$AA?$CI?$AA0?$AAx?$AA?$CF?$AA0?$AA8?$AAx?$AA?9?$AA?$DO?$AA?$CF?$AAd?$AA?1?$AA?$CF?$AAd@ 000155c8     oal:intr.obj
 0001:00004644       ??_C@_1DM@GADKKEEP@?$AA?9?$AAB?$AAS?$AAP?$AAI?$AAn?$AAt?$AAr?$AAE?$AAn?$AAa?$AAb?$AAl?$AAe?$AAI?$AAr?$AAq?$AA?$CI?$AAi?$AAr?$AAq?$AA?5?$AA?$DN?$AA?5?$AA?$CF?$AAd?$AA?$CJ?$AA?$AN?$AA?6?$AA?$AA@ 00015644     oal:intr.obj
 0001:00004680       ??_C@_1DA@PAHKCAOI@?$AA?$CL?$AAB?$AAS?$AAP?$AAI?$AAn?$AAt?$AAr?$AAE?$AAn?$AAa?$AAb?$AAl?$AAe?$AAI?$AAr?$AAq?$AA?$CI?$AA?$CF?$AAd?$AA?$CJ?$AA?$AN?$AA?6?$AA?$AA@ 00015680     oal:intr.obj
 0001:000046b0       ??_C@_1DO@FFIBACGK@?$AA?9?$AAB?$AAS?$AAP?$AAI?$AAn?$AAt?$AAr?$AAD?$AAi?$AAs?$AAa?$AAb?$AAl?$AAe?$AAI?$AAr?$AAq?$AA?$CI?$AAi?$AAr?$AAq?$AA?5?$AA?$DN?$AA?5?$AA?$CF?$AAd?$AA?$CJ?$AA?$AN?$AA?6?$AA?$AA@ 000156b0     oal:intr.obj
 0001:000046f0       ??_C@_1DC@CAJPFJLN@?$AA?$CL?$AAB?$AAS?$AAP?$AAI?$AAn?$AAt?$AAr?$AAD?$AAi?$AAs?$AAa?$AAb?$AAl?$AAe?$AAI?$AAr?$AAq?$AA?$CI?$AA?$CF?$AAd?$AA?$CJ?$AA?$AN?$AA?6?$AA?$AA@ 000156f0     oal:intr.obj
 0001:00004724       ??_C@_1DI@MKBFOAP@?$AA?9?$AAB?$AAS?$AAP?$AAI?$AAn?$AAt?$AAr?$AAD?$AAo?$AAn?$AAe?$AAI?$AAr?$AAq?$AA?$CI?$AAi?$AAr?$AAq?$AA?5?$AA?$DN?$AA?5?$AA?$CF?$AAd?$AA?$CJ?$AA?$AN?$AA?6?$AA?$AA@ 00015724     oal:intr.obj
 0001:0000475c       ??_C@_1CM@KNGKPFDP@?$AA?$CL?$AAB?$AAS?$AAP?$AAI?$AAn?$AAt?$AAr?$AAD?$AAo?$AAn?$AAe?$AAI?$AAr?$AAq?$AA?$CI?$AA?$CF?$AAd?$AA?$CJ?$AA?$AN?$AA?6?$AA?$AA@ 0001575c     oal:intr.obj
 0001:00004788       ??_C@_1DM@JIJHLIGL@?$AA?9?$AAB?$AAS?$AAP?$AAI?$AAn?$AAt?$AAr?$AAA?$AAc?$AAt?$AAi?$AAv?$AAe?$AAI?$AAr?$AAq?$AA?$CI?$AAi?$AAr?$AAq?$AA?5?$AA?$DN?$AA?5?$AA?$CF?$AAd?$AA?$CJ?$AA?$AN?$AA?6?$AA?$AA@ 00015788     oal:intr.obj
 0001:000047c4       ??_C@_1DA@LLHLNMJK@?$AA?$CL?$AAB?$AAS?$AAP?$AAI?$AAn?$AAt?$AAr?$AAA?$AAc?$AAt?$AAi?$AAv?$AAe?$AAI?$AAr?$AAq?$AA?$CI?$AA?$CF?$AAd?$AA?$CJ?$AA?$AN?$AA?6?$AA?$AA@ 000157c4     oal:intr.obj
 0001:000047f4       ??_C@_1O@EPIGJBLB@?$AAA?$AAR?$AAM?$AA9?$AA2?$AA6?$AA?$AA@ 000157f4     oal:ioctl.obj
 0001:00004804       ??_C@_1BK@PCMMEMDD@?$AAT?$AAo?$AAp?$AAa?$AAz?$AA?5?$AAi?$AA?4?$AAM?$AAX?$AA2?$AA5?$AA?$AA@ 00015804     oal:ioctl.obj
 0001:00004820       ??_C@_1CC@PANGHJNL@?$AAD?$AAe?$AAv?$AAi?$AAc?$AAe?$AA?5?$AAS?$AAo?$AAl?$AAu?$AAt?$AAi?$AAo?$AAn?$AAs?$AA?$AA@ 00015820     oal:ioctl.obj
 0001:00004848       ??_C@_1EK@FDOEKKAH@?$AAD?$AAe?$AAv?$AAi?$AAc?$AAe?$AA?5?$AAS?$AAo?$AAl?$AAu?$AAt?$AAi?$AAo?$AAn?$AAs?$AA?5?$AAT?$AAo?$AAp?$AAa?$AAz?$AA?5?$AAi?$AA?4?$AAM?$AAX?$AA2?$AA5?$AA?5?$AAD?$AAe@ 00015848     oal:ioctl.obj
 0001:00004894       ??_C@_1M@PAMBAKIJ@?$AAT?$AAo?$AAp?$AAa?$AAz?$AA?$AA@ 00015894     oal:ioctl.obj
 0001:00004930       g_oalIoCtlTable            00015930     oal:ioctl.obj
 0001:00004ac8       ??_C@_1BO@FIGFABFD@?$AAD?$AAe?$AAf?$AAa?$AAu?$AAl?$AAt?$AAG?$AAa?$AAt?$AAe?$AAw?$AAa?$AAy?$AA?$AA@ 00015ac8     oal:ioctl.obj
 0001:00004ae8       ??_C@_1BG@GEHIKCEG@?$AAS?$AAu?$AAb?$AAn?$AAe?$AAt?$AAm?$AAa?$AAs?$AAk?$AA?$AA@ 00015ae8     oal:ioctl.obj
 0001:00004b00       ??_C@_1BE@FELOAGJB@?$AAI?$AAp?$AAA?$AAd?$AAd?$AAr?$AAe?$AAs?$AAs?$AA?$AA@ 00015b00     oal:ioctl.obj
 0001:00004b14       ??_C@_1BG@GPKEPLMJ@?$AAE?$AAn?$AAa?$AAb?$AAl?$AAe?$AAD?$AAH?$AAC?$AAP?$AA?$AA@ 00015b14     oal:ioctl.obj
 0001:00004b2c       ??_C@_1CM@ENFANCFN@?$AAC?$AAo?$AAm?$AAm?$AA?2?$AAF?$AAE?$AAC?$AA1?$AA?2?$AAP?$AAa?$AAr?$AAm?$AAs?$AA?2?$AAT?$AAc?$AAp?$AAI?$AAp?$AA?$AA@ 00015b2c     oal:ioctl.obj
 0001:00004b58       ??_C@_1BI@JIGNMLMI@?$AAM?$AAA?$AAC?$AAA?$AAd?$AAd?$AAr?$AAe?$AAs?$AAs?$AA3?$AA?$AA@ 00015b58     oal:ioctl.obj
 0001:00004b70       ??_C@_1BI@CANBKMKN@?$AAM?$AAA?$AAC?$AAA?$AAd?$AAd?$AAr?$AAe?$AAs?$AAs?$AA2?$AA?$AA@ 00015b70     oal:ioctl.obj
 0001:00004b88       ??_C@_1BI@DCGEADED@?$AAM?$AAA?$AAC?$AAA?$AAd?$AAd?$AAr?$AAe?$AAs?$AAs?$AA1?$AA?$AA@ 00015b88     oal:ioctl.obj
 0001:00004ba0       ??_C@_1CA@MLFPFCIF@?$AAC?$AAo?$AAm?$AAm?$AA?2?$AAF?$AAE?$AAC?$AA1?$AA?2?$AAP?$AAa?$AAr?$AAm?$AAs?$AA?$AA@ 00015ba0     oal:ioctl.obj
 0001:00004bc0       ??_C@_1GC@FLMGGHIP@?$AAC?$AAs?$AAp?$AAi?$AAM?$AAa?$AAs?$AAt?$AAe?$AAr?$AAD?$AAa?$AAt?$AAa?$AAE?$AAx?$AAc?$AAh?$AAa?$AAn?$AAg?$AAe?$AA?3?$AA?5?$AA?5?$AAu?$AAn?$AAs?$AAu?$AAp?$AAp?$AAo@ 00015bc0     oal:ioctl.obj
 0001:00004c24       ??_C@_1DK@IMDDFKCB@?$AAD?$AAu?$AAm?$AAp?$AAC?$AAs?$AAp?$AAi?$AAR?$AAe?$AAg?$AAs?$AA?5?$AAT?$AAX?$AAD?$AAA?$AAT?$AAA?$AA?5?$AA?$DN?$AA?5?$AA0?$AAx?$AA?$CF?$AAx?$AA?$AN?$AA?6?$AA?$AA@ 00015c24     oal:ioctl.obj
 0001:00004c60       ??_C@_1DM@LGHBBFDO@?$AAD?$AAu?$AAm?$AAp?$AAC?$AAs?$AAp?$AAi?$AAR?$AAe?$AAg?$AAs?$AA?5?$AAT?$AAE?$AAS?$AAT?$AAR?$AAE?$AAG?$AA?5?$AA?$DN?$AA?5?$AA0?$AAx?$AA?$CF?$AAx?$AA?$AN?$AA?6?$AA?$AA@ 00015c60     oal:ioctl.obj
 0001:00004c9c       ??_C@_1DM@KNFADDON@?$AAD?$AAu?$AAm?$AAp?$AAC?$AAs?$AAp?$AAi?$AAR?$AAe?$AAg?$AAs?$AA?5?$AAS?$AAT?$AAA?$AAT?$AAR?$AAE?$AAG?$AA?5?$AA?$DN?$AA?5?$AA0?$AAx?$AA?$CF?$AAx?$AA?$AN?$AA?6?$AA?$AA@ 00015c9c     oal:ioctl.obj
 0001:00004cd8       ??_C@_1DK@MFHMENBO@?$AAD?$AAu?$AAm?$AAp?$AAC?$AAs?$AAp?$AAi?$AAR?$AAe?$AAg?$AAs?$AA?5?$AAR?$AAX?$AAD?$AAA?$AAT?$AAA?$AA?5?$AA?$DN?$AA?5?$AA0?$AAx?$AA?$CF?$AAx?$AA?$AN?$AA?6?$AA?$AA@ 00015cd8     oal:ioctl.obj
 0001:00004d18       ??_C@_1EA@HLDHIFIA@?$AAD?$AAu?$AAm?$AAp?$AAC?$AAs?$AAp?$AAi?$AAR?$AAe?$AAg?$AAs?$AA?5?$AAP?$AAE?$AAR?$AAI?$AAO?$AAD?$AAR?$AAE?$AAG?$AA?5?$AA?$DN?$AA?5?$AA0?$AAx?$AA?$CF?$AAx?$AA?$AN?$AA?6?$AA?$AA@ 00015d18     oal:ioctl.obj
 0001:00004d58       ??_C@_1DK@MEGFEOOE@?$AAD?$AAu?$AAm?$AAp?$AAC?$AAs?$AAp?$AAi?$AAR?$AAe?$AAg?$AAs?$AA?5?$AAI?$AAN?$AAT?$AAR?$AAE?$AAG?$AA?5?$AA?$DN?$AA?5?$AA0?$AAx?$AA?$CF?$AAx?$AA?$AN?$AA?6?$AA?$AA@ 00015d58     oal:ioctl.obj
 0001:00004d94       ??_C@_1DK@PPLNJIJB@?$AAD?$AAu?$AAm?$AAp?$AAC?$AAs?$AAp?$AAi?$AAR?$AAe?$AAg?$AAs?$AA?5?$AAD?$AAM?$AAA?$AAR?$AAE?$AAG?$AA?5?$AA?$DN?$AA?5?$AA0?$AAx?$AA?$CF?$AAx?$AA?$AN?$AA?6?$AA?$AA@ 00015d94     oal:ioctl.obj
 0001:00004dd0       ??_C@_1DK@DGEPFHKP@?$AAD?$AAu?$AAm?$AAp?$AAC?$AAs?$AAp?$AAi?$AAR?$AAe?$AAg?$AAs?$AA?5?$AAC?$AAO?$AAN?$AAR?$AAE?$AAG?$AA?5?$AA?$DN?$AA?5?$AA0?$AAx?$AA?$CF?$AAx?$AA?$AN?$AA?6?$AA?$AA@ 00015dd0     oal:ioctl.obj
 0001:00004e0c       ??_C@_1BO@CPNGNHGD@?$AAD?$AAu?$AAm?$AAp?$AAC?$AAs?$AAp?$AAi?$AAR?$AAe?$AAg?$AAs?$AA?$AN?$AA?6?$AA?$AA@ 00015e0c     oal:ioctl.obj
 0001:00004f50       ??_C@_1EK@CACKHHPA@?$AAI?$AAn?$AAv?$AAa?$AAl?$AAi?$AAd?$AA?5?$AAp?$AAr?$AAo?$AAf?$AAi?$AAl?$AAe?$AAr?$AA?5?$AAc?$AAl?$AAo?$AAc?$AAk?$AA?5?$AAs?$AAo?$AAu?$AAr?$AAc?$AAe?$AA?5?$AA?3?$AA?5@ 00015f50     oal:profiler.obj
 0001:00005030       ??_C@_1DO@JHJONFOE@?$AA?9?$AAO?$AAA?$AAL?$AAI?$AAo?$AAC?$AAt?$AAl?$AAH?$AAa?$AAl?$AAD?$AAd?$AAk?$AAC?$AAa?$AAl?$AAl?$AA?$CI?$AAr?$AAc?$AA?5?$AA?$DN?$AA?5?$AA?$CF?$AAd?$AA?$CJ?$AA?$AN?$AA?6?$AA?$AA@ 00016030     oal_io:ioctl.obj
 0001:00005070       ??_C@_1HM@DONGDDHM@?$AAE?$AAR?$AAR?$AAO?$AAR?$AA?3?$AA?5?$AAO?$AAA?$AAL?$AAI?$AAo?$AAc?$AAt?$AAl?$AAH?$AAa?$AAl?$AAD?$AAd?$AAk?$AAC?$AAa?$AAl?$AAl?$AA?3?$AA?5?$AAU?$AAn?$AAs?$AAu?$AAp@ 00016070     oal_io:ioctl.obj
 0001:000050f0       ??_C@_1GE@BFODAIDF@?$AAE?$AAR?$AAR?$AAO?$AAR?$AA?3?$AA?5?$AAO?$AAA?$AAL?$AAI?$AAo?$AAc?$AAt?$AAl?$AAH?$AAa?$AAl?$AAD?$AAd?$AAk?$AAC?$AAa?$AAl?$AAl?$AA?3?$AA?5?$AAU?$AAn?$AAs?$AAu?$AAp@ 000160f0     oal_io:ioctl.obj
 0001:00005158       ??_C@_1FM@IFHLCDE@?$AAE?$AAR?$AAR?$AAO?$AAR?$AA?3?$AAO?$AAA?$AAL?$AAI?$AAo?$AAc?$AAt?$AAl?$AAH?$AAa?$AAl?$AAD?$AAd?$AAk?$AAC?$AAa?$AAl?$AAl?$AA?3?$AA?5?$AAI?$AAN?$AAV?$AAA?$AAL?$AAI@ 00016158     oal_io:ioctl.obj
 0001:000051b4       ??_C@_1DG@HOFDDFMH@?$AA?$CL?$AAO?$AAA?$AAL?$AAI?$AAo?$AAC?$AAt?$AAl?$AAH?$AAa?$AAl?$AAD?$AAd?$AAk?$AAC?$AAa?$AAl?$AAl?$AA?$CI?$AA?4?$AA?4?$AA?4?$AA?$CJ?$AA?$AN?$AA?6?$AA?$AA@ 000161b4     oal_io:ioctl.obj
 0001:00005280       ??_C@_1DK@DKAHFGMP@?$AA?9?$AAO?$AAA?$AAL?$AAI?$AAo?$AAB?$AAu?$AAs?$AAP?$AAo?$AAw?$AAe?$AAr?$AAO?$AAf?$AAf?$AA?$CI?$AAr?$AAc?$AA?5?$AA?$DN?$AA?5?$AA?$CF?$AAd?$AA?$CJ?$AA?$AN?$AA?6?$AA?$AA@ 00016280     oal_io:power.obj
 0001:000052bc       ??_C@_1DI@PEAMECNB@?$AA?$CL?$AAO?$AAA?$AAL?$AAI?$AAo?$AAB?$AAu?$AAs?$AAP?$AAo?$AAw?$AAe?$AAr?$AAO?$AAf?$AAf?$AA?$CI?$AA?$CF?$AAd?$AA?0?$AA?5?$AA?$CF?$AAd?$AA?$CJ?$AA?$AN?$AA?6?$AA?$AA@ 000162bc     oal_io:power.obj
 0001:000052f4       ??_C@_1DI@BEKMCAGI@?$AA?9?$AAO?$AAA?$AAL?$AAI?$AAo?$AAB?$AAu?$AAs?$AAP?$AAo?$AAw?$AAe?$AAr?$AAO?$AAn?$AA?$CI?$AAr?$AAc?$AA?5?$AA?$DN?$AA?5?$AA?$CF?$AAd?$AA?$CJ?$AA?$AN?$AA?6?$AA?$AA@ 000162f4     oal_io:power.obj
 0001:0000532c       ??_C@_1DG@BNAKMMEE@?$AA?$CL?$AAO?$AAA?$AAL?$AAI?$AAo?$AAB?$AAu?$AAs?$AAP?$AAo?$AAw?$AAe?$AAr?$AAO?$AAn?$AA?$CI?$AA?$CF?$AAd?$AA?0?$AA?5?$AA?$CF?$AAd?$AA?$CJ?$AA?$AN?$AA?6?$AA?$AA@ 0001632c     oal_io:power.obj
 0001:000053f8       ??_C@_1KE@FCFGNLKM@?$AA?9?$AAO?$AAA?$AAL?$AAT?$AAr?$AAa?$AAn?$AAs?$AAl?$AAa?$AAt?$AAe?$AAB?$AAu?$AAs?$AAA?$AAd?$AAd?$AAr?$AAe?$AAs?$AAs?$AA?$CI?$AAa?$AAd?$AAd?$AAr?$AAe?$AAs?$AAs?$AAS@ 000163f8     oal_io:trans.obj
 0001:000054a0       ??_C@_1GI@BPOGFGAB@?$AA?$CL?$AAO?$AAA?$AAL?$AAI?$AAo?$AAT?$AAr?$AAa?$AAn?$AAs?$AAl?$AAa?$AAt?$AAe?$AAB?$AAu?$AAs?$AAA?$AAd?$AAd?$AAr?$AAe?$AAs?$AAs?$AA?$CI?$AA?$CF?$AAd?$AA?0?$AA?5?$AA?$CF?$AAd@ 000164a0     oal_io:trans.obj
 0001:00005508       ??_C@_1HM@IKCJOCJL@?$AA?9?$AAO?$AAA?$AAL?$AAT?$AAr?$AAa?$AAn?$AAs?$AAl?$AAa?$AAt?$AAe?$AAS?$AAy?$AAs?$AAt?$AAe?$AAm?$AAA?$AAd?$AAd?$AAr?$AAe?$AAs?$AAs?$AA?$CI?$AAb?$AAu?$AAs?$AAA?$AAd@ 00016508     oal_io:trans.obj
 0001:00005588       ??_C@_1GC@GKDDBMML@?$AA?$CL?$AAO?$AAA?$AAL?$AAT?$AAr?$AAa?$AAn?$AAs?$AAl?$AAa?$AAt?$AAe?$AAS?$AAy?$AAs?$AAt?$AAe?$AAm?$AAA?$AAd?$AAd?$AAr?$AAe?$AAs?$AAs?$AA?$CI?$AA?$CF?$AAd?$AA?0?$AA?5?$AA?$CF@ 00016588     oal_io:trans.obj
 0001:00005680       ??_C@_1EM@KGGHBFBJ@?$AA?$CL?$AAO?$AAA?$AAL?$AAI?$AAo?$AAC?$AAt?$AAl?$AAH?$AAa?$AAl?$AAR?$AAe?$AAq?$AAu?$AAe?$AAs?$AAt?$AAS?$AAy?$AAs?$AAI?$AAn?$AAt?$AAr?$AA?$CI?$AAr?$AAc?$AA?5?$AA?$DN?$AA?5@ 00016680     oal_intr_mx25_topaz_v1:ioctl.obj
 0001:000056d0       ??_C@_1GK@HKEIPOOO@?$AAW?$AAA?$AAR?$AAN?$AA?3?$AA?5?$AAI?$AAO?$AAC?$AAT?$AAL?$AA_?$AAH?$AAA?$AAL?$AA_?$AAR?$AAE?$AAQ?$AAU?$AAE?$AAS?$AAT?$AA_?$AAS?$AAY?$AAS?$AAI?$AAN?$AAT?$AAR?$AA?5@ 000166d0     oal_intr_mx25_topaz_v1:ioctl.obj
 0001:0000573c       ??_C@_1DK@BMKLIPKJ@?$AA?$CL?$AAO?$AAA?$AAL?$AAI?$AAo?$AAC?$AAt?$AAl?$AAH?$AAa?$AAl?$AAR?$AAe?$AAq?$AAu?$AAe?$AAs?$AAt?$AAS?$AAy?$AAs?$AAI?$AAn?$AAt?$AAr?$AA?$AN?$AA?6?$AA?$AA@ 0001673c     oal_intr_mx25_topaz_v1:ioctl.obj
 0001:00005778       ??_C@_1GK@LIJAJEGD@?$AAW?$AAA?$AAR?$AAN?$AA?3?$AA?5?$AAI?$AAO?$AAC?$AAT?$AAL?$AA_?$AAH?$AAA?$AAL?$AA_?$AAR?$AAE?$AAL?$AAE?$AAA?$AAS?$AAE?$AA_?$AAS?$AAY?$AAS?$AAI?$AAN?$AAT?$AAR?$AA?5@ 00016778     oal_intr_mx25_topaz_v1:ioctl.obj
 0001:000057e8       ??_C@_1EM@DFAKLPBP@?$AA?9?$AAO?$AAA?$AAL?$AAI?$AAo?$AAC?$AAt?$AAl?$AAH?$AAa?$AAl?$AAR?$AAe?$AAq?$AAu?$AAe?$AAs?$AAt?$AAS?$AAy?$AAs?$AAI?$AAn?$AAt?$AAr?$AA?$CI?$AAr?$AAc?$AA?5?$AA?$DN?$AA?5@ 000167e8     oal_intr_mx25_topaz_v1:ioctl.obj
 0001:00005838       ??_C@_1GC@BACPHDPH@?$AAW?$AAA?$AAR?$AAN?$AA?3?$AA?5?$AAI?$AAO?$AAC?$AAT?$AAL?$AA_?$AAH?$AAA?$AAL?$AA_?$AAR?$AAE?$AAQ?$AAU?$AAE?$AAS?$AAT?$AA_?$AAI?$AAR?$AAQ?$AA?5?$AAi?$AAn?$AAv?$AAa@ 00016838     oal_intr_mx25_topaz_v1:ioctl.obj
 0001:0000589c       ??_C@_1DC@DIKJBBIL@?$AA?$CL?$AAO?$AAA?$AAL?$AAI?$AAo?$AAC?$AAt?$AAl?$AAH?$AAa?$AAl?$AAR?$AAe?$AAq?$AAu?$AAe?$AAs?$AAt?$AAI?$AAr?$AAq?$AA?$AN?$AA?6?$AA?$AA@ 0001689c     oal_intr_mx25_topaz_v1:ioctl.obj
 0001:00005960       ??_C@_1IG@BENIAHFO@?$AAE?$AAR?$AAR?$AAO?$AAR?$AA?3?$AA?5?$AAO?$AAA?$AAL?$AAI?$AAo?$AAC?$AAt?$AAl?$AAH?$AAa?$AAl?$AAU?$AAp?$AAd?$AAa?$AAt?$AAe?$AAM?$AAo?$AAd?$AAe?$AA?3?$AA?5?$AAD?$AAe@ 00016960     oal_ioctl_mx25_topaz_v1:imgupd.obj
 0001:000059e8       ??_C@_1GK@GKDOOKDE@?$AAE?$AAR?$AAR?$AAO?$AAR?$AA?3?$AA?5?$AAO?$AAA?$AAL?$AAI?$AAo?$AAC?$AAt?$AAl?$AAH?$AAa?$AAl?$AAU?$AAp?$AAd?$AAa?$AAt?$AAe?$AAM?$AAo?$AAd?$AAe?$AA?3?$AA?5?$AAI?$AAn@ 000169e8     oal_ioctl_mx25_topaz_v1:imgupd.obj
 0001:00005ae8       ??_C@_1FA@KIKMJANO@?$AA?9?$AAO?$AAA?$AAL?$AAI?$AAo?$AAC?$AAt?$AAl?$AAH?$AAa?$AAl?$AAG?$AAe?$AAt?$AAR?$AAe?$AAg?$AAS?$AAe?$AAc?$AAu?$AAr?$AAe?$AAK?$AAe?$AAy?$AAs?$AA?$CI?$AAr?$AAc?$AA?5@ 00016ae8     oal_ioctl_mx25_topaz_v1:securekeys.obj
 0001:00005bc8       ??_C@_1EE@LLJFHFAM@?$AA?9?$AAO?$AAA?$AAL?$AAI?$AAo?$AAC?$AAt?$AAl?$AAP?$AAr?$AAo?$AAc?$AAe?$AAs?$AAs?$AAo?$AAr?$AAI?$AAn?$AAf?$AAo?$AA?$CI?$AAr?$AAc?$AA?5?$AA?$DN?$AA?5?$AA?$CF?$AAd?$AA?$CJ?$AA?$AN@ 00016bc8     oal_ioctl_mx25_topaz_v1:procinfo.obj
 0001:00005c10       ??_C@_1GI@EFCEJCLG@?$AAE?$AAR?$AAR?$AAO?$AAR?$AA?3?$AAO?$AAA?$AAL?$AAI?$AAo?$AAC?$AAt?$AAl?$AAP?$AAr?$AAo?$AAc?$AAe?$AAs?$AAs?$AAo?$AAr?$AAI?$AAn?$AAf?$AAo?$AA?3?$AA?5?$AAV?$AAe?$AAn@ 00016c10     oal_ioctl_mx25_topaz_v1:procinfo.obj
 0001:00005c78       ??_C@_1GE@JPAPEENG@?$AAE?$AAR?$AAR?$AAO?$AAR?$AA?3?$AAO?$AAA?$AAL?$AAI?$AAo?$AAC?$AAt?$AAl?$AAP?$AAr?$AAo?$AAc?$AAe?$AAs?$AAs?$AAo?$AAr?$AAI?$AAn?$AAf?$AAo?$AA?3?$AA?5?$AAN?$AAa?$AAm@ 00016c78     oal_ioctl_mx25_topaz_v1:procinfo.obj
 0001:00005ce0       ??_C@_1GE@OFFJPJMM@?$AAE?$AAR?$AAR?$AAO?$AAR?$AA?3?$AAO?$AAA?$AAL?$AAI?$AAo?$AAC?$AAt?$AAl?$AAP?$AAr?$AAo?$AAc?$AAe?$AAs?$AAs?$AAo?$AAr?$AAI?$AAn?$AAf?$AAo?$AA?3?$AA?5?$AAC?$AAo?$AAr@ 00016ce0     oal_ioctl_mx25_topaz_v1:procinfo.obj
 0001:00005d48       ??_C@_1GA@EACFLEMI@?$AAW?$AAA?$AAR?$AAN?$AA?3?$AA?5?$AAO?$AAA?$AAL?$AAI?$AAo?$AAC?$AAt?$AAl?$AAP?$AAr?$AAo?$AAc?$AAe?$AAs?$AAs?$AAo?$AAr?$AAI?$AAn?$AAf?$AAo?$AA?3?$AA?5?$AAB?$AAu?$AAf@ 00016d48     oal_ioctl_mx25_topaz_v1:procinfo.obj
 0001:00005da8       ??_C@_1GK@MJNAOGCM@?$AAW?$AAA?$AAR?$AAN?$AA?3?$AA?5?$AAO?$AAA?$AAL?$AAI?$AAo?$AAC?$AAt?$AAl?$AAP?$AAr?$AAo?$AAc?$AAe?$AAs?$AAs?$AAo?$AAr?$AAI?$AAn?$AAf?$AAo?$AA?3?$AA?5?$AAI?$AAn?$AAv@ 00016da8     oal_ioctl_mx25_topaz_v1:procinfo.obj
 0001:00005e14       ??_C@_1DM@NEACNOML@?$AA?$CL?$AAO?$AAA?$AAL?$AAI?$AAo?$AAC?$AAt?$AAl?$AAP?$AAr?$AAo?$AAc?$AAe?$AAs?$AAs?$AAo?$AAr?$AAI?$AAn?$AAf?$AAo?$AA?$CI?$AA?4?$AA?4?$AA?4?$AA?$CJ?$AA?$AN?$AA?6?$AA?$AA@ 00016e14     oal_ioctl_mx25_topaz_v1:procinfo.obj
 0001:00005ef0       ??_C@_1NA@DANHDCDJ@?$AAW?$AAa?$AAr?$AAn?$AAi?$AAn?$AAg?$AA?3?$AA?5?$AAI?$AAO?$AAC?$AAT?$AAL?$AA_?$AAH?$AAA?$AAL?$AA_?$AAG?$AAE?$AAT?$AA_?$AAU?$AAU?$AAI?$AAD?$AA?5?$AAi?$AAs?$AA?5?$AAu@ 00016ef0     oal_ioctl_mx25_topaz_v1:uuid.obj
 0001:00005fc0       ??_C@_1HC@GCDGDEMK@?$AAE?$AAR?$AAR?$AAO?$AAR?$AA?3?$AA?5?$AAO?$AAA?$AAL?$AAI?$AAo?$AAC?$AAt?$AAl?$AAH?$AAa?$AAl?$AAG?$AAe?$AAt?$AAU?$AAU?$AAI?$AAD?$AA?3?$AA?5?$AAD?$AAe?$AAv?$AAi?$AAc@ 00016fc0     oal_ioctl_mx25_topaz_v1:uuid.obj
 0001:00006038       ??_C@_1FK@JJDHOCFD@?$AAW?$AAA?$AAR?$AAN?$AA?3?$AA?5?$AAO?$AAA?$AAL?$AAI?$AAo?$AAC?$AAt?$AAl?$AAH?$AAa?$AAl?$AAG?$AAe?$AAt?$AAU?$AAU?$AAI?$AAD?$AA?3?$AA?5?$AAB?$AAu?$AAf?$AAf?$AAe?$AAr@ 00017038     oal_ioctl_mx25_topaz_v1:uuid.obj
 0001:00006098       ??_C@_1GE@PBBGNNAO@?$AAW?$AAA?$AAR?$AAN?$AA?3?$AA?5?$AAO?$AAA?$AAL?$AAI?$AAo?$AAC?$AAt?$AAl?$AAH?$AAa?$AAl?$AAG?$AAe?$AAt?$AAU?$AAU?$AAI?$AAD?$AA?3?$AA?5?$AAI?$AAn?$AAv?$AAa?$AAl?$AAi@ 00017098     oal_ioctl_mx25_topaz_v1:uuid.obj
 0001:00006100       ??_C@_1OE@KFAEFCPB@?$AAW?$AAa?$AAr?$AAn?$AAi?$AAn?$AAg?$AA?3?$AA?5?$AAy?$AAo?$AAu?$AA?5?$AAa?$AAr?$AAe?$AA?5?$AAc?$AAa?$AAl?$AAl?$AAi?$AAn?$AAg?$AA?5?$AAI?$AAO?$AAC?$AAT?$AAL?$AA_?$AAH@ 00017100     oal_ioctl_mx25_topaz_v1:uuid.obj
 0001:00006200       ??_C@_1FO@DMDJMEMA@?$AA?9?$AAO?$AAA?$AAL?$AAI?$AAo?$AAC?$AAt?$AAl?$AAH?$AAa?$AAl?$AAG?$AAe?$AAt?$AAD?$AAe?$AAv?$AAi?$AAc?$AAe?$AAI?$AAn?$AAf?$AAo?$AA?$CI?$AAS?$AAP?$AAI?$AA?5?$AA?$DN?$AA?5@ 00017200     oal_ioctl_mx25_topaz_v1:deviceinfo.obj
 0001:00006260       ??_C@_1GG@BAANNGGI@?$AAE?$AAR?$AAR?$AAO?$AAR?$AA?3?$AA?5?$AAO?$AAA?$AAL?$AAI?$AAo?$AAC?$AAt?$AAl?$AAH?$AAa?$AAl?$AAG?$AAe?$AAt?$AAD?$AAe?$AAv?$AAi?$AAc?$AAe?$AAI?$AAn?$AAf?$AAo?$AA?3@ 00017260     oal_ioctl_mx25_topaz_v1:deviceinfo.obj
 0001:000062c8       ??_C@_1GK@FDHCLEBC@?$AAE?$AAR?$AAR?$AAO?$AAR?$AA?3?$AA?5?$AAO?$AAA?$AAL?$AAI?$AAo?$AAC?$AAt?$AAl?$AAH?$AAa?$AAl?$AAG?$AAe?$AAt?$AAD?$AAe?$AAv?$AAi?$AAc?$AAe?$AAI?$AAn?$AAf?$AAo?$AA?3@ 000172c8     oal_ioctl_mx25_topaz_v1:deviceinfo.obj
 0001:00006338       ??_C@_1EC@NLAFOPGI@?$AA?$CL?$AAO?$AAA?$AAL?$AAI?$AAo?$AAC?$AAt?$AAl?$AAH?$AAa?$AAl?$AAG?$AAe?$AAt?$AAD?$AAe?$AAv?$AAi?$AAc?$AAe?$AAI?$AAn?$AAf?$AAo?$AA?$CI?$AA?4?$AA?4?$AA?4?$AA?$CJ?$AA?$AN?$AA?6@ 00017338     oal_ioctl_mx25_topaz_v1:deviceinfo.obj
 0001:0000637c       ??_C@_11LOCGONAA@?$AA?$AA@ 0001737c     oal_ioctl_mx25_topaz_v1:deviceinfo.obj
 0001:00006380       ??_C@_1BEM@IMHNFGHE@?$AAW?$AAa?$AAr?$AAn?$AAi?$AAn?$AAg?$AA?3?$AA?5?$AAy?$AAo?$AAu?$AA?5?$AAa?$AAr?$AAe?$AA?5?$AAr?$AAe?$AAq?$AAu?$AAe?$AAs?$AAt?$AAi?$AAn?$AAg?$AA?5?$AAI?$AAO?$AAC?$AAT@ 00017380     oal_ioctl_mx25_topaz_v1:deviceinfo.obj
 0001:000064cc       ??_C@_1CI@DNLIPKLH@?$AAS?$AAP?$AAI?$AA_?$AAG?$AAE?$AAT?$AAP?$AAL?$AAA?$AAT?$AAF?$AAO?$AAR?$AAM?$AAT?$AAY?$AAP?$AAE?$AA?$AA@ 000174cc     oal_ioctl_mx25_topaz_v1:deviceinfo.obj
 0001:000064f4       ??_C@_1BO@MIPEKPNN@?$AAS?$AAP?$AAI?$AA_?$AAG?$AAE?$AAT?$AAO?$AAE?$AAM?$AAI?$AAN?$AAF?$AAO?$AA?$AA@ 000174f4     oal_ioctl_mx25_topaz_v1:deviceinfo.obj
 0001:00006514       ??_C@_1CO@EPEFNCOE@?$AAS?$AAP?$AAI?$AA_?$AAG?$AAE?$AAT?$AAP?$AAL?$AAA?$AAT?$AAF?$AAO?$AAR?$AAM?$AAV?$AAE?$AAR?$AAS?$AAI?$AAO?$AAN?$AA?$AA@ 00017514     oal_ioctl_mx25_topaz_v1:deviceinfo.obj
 0001:00006544       ??_C@_1CG@NCDPNLLL@?$AAS?$AAP?$AAI?$AA_?$AAG?$AAE?$AAT?$AAP?$AAR?$AAO?$AAJ?$AAE?$AAC?$AAT?$AAN?$AAA?$AAM?$AAE?$AA?$AA@ 00017544     oal_ioctl_mx25_topaz_v1:deviceinfo.obj
 0001:0000656c       ??_C@_1CI@BNCCNAEN@?$AAS?$AAP?$AAI?$AA_?$AAG?$AAE?$AAT?$AAP?$AAL?$AAA?$AAT?$AAF?$AAO?$AAR?$AAM?$AAN?$AAA?$AAM?$AAE?$AA?$AA@ 0001756c     oal_ioctl_mx25_topaz_v1:deviceinfo.obj
 0001:00006594       ??_C@_1CE@JLAPMINP@?$AAS?$AAP?$AAI?$AA_?$AAG?$AAE?$AAT?$AAB?$AAO?$AAO?$AAT?$AAM?$AAE?$AAN?$AAA?$AAM?$AAE?$AA?$AA@ 00017594     oal_ioctl_mx25_topaz_v1:deviceinfo.obj
 0001:000065b8       ??_C@_1BI@MGABGHAL@?$AAS?$AAP?$AAI?$AA_?$AAG?$AAE?$AAT?$AAU?$AAU?$AAI?$AAD?$AA?$AA@ 000175b8     oal_ioctl_mx25_topaz_v1:deviceinfo.obj
 0001:000065e0       ??_C@_1CG@IIMMCNFM@?$AAS?$AAP?$AAI?$AA_?$AAG?$AAE?$AAT?$AAG?$AAU?$AAI?$AAD?$AAP?$AAA?$AAT?$AAT?$AAE?$AAR?$AAN?$AA?$AA@ 000175e0     oal_ioctl_mx25_topaz_v1:deviceinfo.obj
 0001:00006608       ??_C@_1GO@GEFDPJAG@?$AAW?$AAA?$AAR?$AAN?$AA?3?$AA?5?$AAO?$AAA?$AAL?$AAI?$AAo?$AAC?$AAt?$AAl?$AAH?$AAa?$AAl?$AAG?$AAe?$AAt?$AAD?$AAe?$AAv?$AAi?$AAc?$AAe?$AAi?$AAn?$AAf?$AAo?$AA?3?$AA?3@ 00017608     oal_ioctl_mx25_topaz_v1:deviceinfo.obj
 0001:00006678       ??_C@_1NG@HBFOMIME@?$AAE?$AAR?$AAR?$AAO?$AAR?$AA?3?$AA?5?$AAO?$AAA?$AAL?$AAI?$AAo?$AAC?$AAt?$AAl?$AAH?$AAa?$AAl?$AAG?$AAe?$AAt?$AAD?$AAe?$AAv?$AAi?$AAc?$AAe?$AAi?$AAn?$AAf?$AAo?$AA?3@ 00017678     oal_ioctl_mx25_topaz_v1:deviceinfo.obj
 0001:00006750       ??_C@_1LA@BNOICHNN@?$AAE?$AAR?$AAR?$AAO?$AAR?$AA?3?$AA?5?$AAO?$AAA?$AAL?$AAI?$AAo?$AAC?$AAt?$AAl?$AAH?$AAa?$AAl?$AAG?$AAe?$AAt?$AAD?$AAe?$AAv?$AAi?$AAc?$AAe?$AAI?$AAn?$AAf?$AAo?$AA?3@ 00017750     oal_ioctl_mx25_topaz_v1:deviceinfo.obj
 0001:00006890       ??_C@_1EG@HKOJPLNE@?$AA?9?$AAO?$AAA?$AAL?$AAI?$AAo?$AAC?$AAt?$AAl?$AAH?$AAa?$AAl?$AAG?$AAe?$AAt?$AAD?$AAe?$AAv?$AAi?$AAc?$AAe?$AAI?$AAD?$AA?$CI?$AAr?$AAc?$AA?5?$AA?$DN?$AA?5?$AA?$CF?$AAd?$AA?$CJ@ 00017890     oal_ioctl_mx25_topaz_v1:deviceid.obj
 0001:000068d8       ??_C@_1GE@GPJLHAFO@?$AAW?$AAA?$AAR?$AAN?$AA?3?$AA?5?$AAO?$AAA?$AAL?$AAI?$AAo?$AAC?$AAt?$AAl?$AAH?$AAa?$AAl?$AAG?$AAe?$AAt?$AAD?$AAe?$AAv?$AAi?$AAc?$AAe?$AAI?$AAD?$AA?3?$AA?5?$AAI?$AAn@ 000178d8     oal_ioctl_mx25_topaz_v1:deviceid.obj
 0001:00006940       ??_C@_1LK@FOLPDAJB@?$AAW?$AAA?$AAR?$AAN?$AA?3?$AA?5?$AAO?$AAA?$AAL?$AAI?$AAo?$AAC?$AAt?$AAl?$AAH?$AAa?$AAl?$AAG?$AAe?$AAt?$AAD?$AAe?$AAv?$AAi?$AAc?$AAe?$AAI?$AAD?$AA?3?$AA?5?$AAC?$AAa@ 00017940     oal_ioctl_mx25_topaz_v1:deviceid.obj
 0001:00006a00       ??_C@_1LO@DFJMJCEI@?$AAW?$AAA?$AAR?$AAN?$AA?3?$AA?5?$AAO?$AAA?$AAL?$AAI?$AAo?$AAC?$AAt?$AAl?$AAH?$AAa?$AAl?$AAG?$AAe?$AAt?$AAD?$AAe?$AAv?$AAi?$AAc?$AAe?$AAI?$AAD?$AA?3?$AA?5?$AAC?$AAa@ 00017a00     oal_ioctl_mx25_topaz_v1:deviceid.obj
 0001:00006ac0       ??_C@_1PC@IHJIIKFF@?$AAW?$AAa?$AAr?$AAn?$AAi?$AAn?$AAg?$AA?3?$AA?5?$AAy?$AAo?$AAu?$AA?5?$AAa?$AAr?$AAe?$AA?5?$AAr?$AAe?$AAq?$AAu?$AAe?$AAs?$AAt?$AAi?$AAn?$AAg?$AA?5?$AAI?$AAO?$AAC?$AAT@ 00017ac0     oal_ioctl_mx25_topaz_v1:deviceid.obj
 0001:00006bb4       ??_C@_1DO@MLDPBFAO@?$AA?$CL?$AAO?$AAA?$AAL?$AAI?$AAo?$AAc?$AAt?$AAl?$AAH?$AAa?$AAl?$AAG?$AAe?$AAt?$AAD?$AAe?$AAv?$AAi?$AAc?$AAe?$AAI?$AAD?$AA?$CI?$AA?4?$AA?4?$AA?4?$AA?$CJ?$AA?$AN?$AA?6?$AA?$AA@ 00017bb4     oal_ioctl_mx25_topaz_v1:deviceid.obj
 0001:00006c88       ??_C@_1CK@LAAGFJIK@?$AA?$CL?$AAO?$AAA?$AAL?$AAI?$AAo?$AAC?$AAt?$AAl?$AAH?$AAa?$AAl?$AAR?$AAe?$AAb?$AAo?$AAo?$AAt?$AA?$AN?$AA?6?$AA?$AA@ 00017c88     oal_ioctl_mx25_topaz_v1:reboot.obj
 0001:00006d48       ??_C@_1EG@PJLICJDP@?$AA?$CL?$AAO?$AAA?$AAL?$AAI?$AAo?$AAC?$AAt?$AAl?$AAH?$AAa?$AAl?$AAI?$AAr?$AAq?$AA2?$AAS?$AAy?$AAs?$AAi?$AAn?$AAt?$AAr?$AA?$CI?$AAr?$AAc?$AA?5?$AA?$DN?$AA?5?$AA?$CF?$AAd?$AA?$CJ@ 00017d48     oal_ioctl_mx25_topaz_v1:soc_ioctl.obj
 0001:00006d90       ??_C@_1GC@IHFCBEA@?$AAW?$AAA?$AAR?$AAN?$AA?3?$AA?5?$AAI?$AAO?$AAC?$AAT?$AAL?$AA_?$AAH?$AAA?$AAL?$AA_?$AAI?$AAR?$AAQ?$AA2?$AAS?$AAY?$AAS?$AAI?$AAN?$AAT?$AAR?$AA?5?$AAi?$AAn?$AAv?$AAa@ 00017d90     oal_ioctl_mx25_topaz_v1:soc_ioctl.obj
 0001:00006df4       ??_C@_1DE@MPBNEBBN@?$AA?$CL?$AAO?$AAA?$AAL?$AAI?$AAo?$AAC?$AAt?$AAl?$AAH?$AAa?$AAl?$AAI?$AAr?$AAq?$AA2?$AAS?$AAy?$AAs?$AAi?$AAn?$AAt?$AAr?$AA?$AN?$AA?6?$AA?$AA@ 00017df4     oal_ioctl_mx25_topaz_v1:soc_ioctl.obj
 0001:00006e28       ??_C@_1EA@PFPFPLIM@?$AA?$CL?$AAO?$AAA?$AAL?$AAI?$AAo?$AAC?$AAt?$AAl?$AAH?$AAa?$AAl?$AAF?$AAo?$AAr?$AAc?$AAe?$AAI?$AAr?$AAq?$AA?$CI?$AAr?$AAc?$AA?5?$AA?$DN?$AA?5?$AA?$CF?$AAd?$AA?$CJ?$AA?$AN?$AA?6?$AA?$AA@ 00017e28     oal_ioctl_mx25_topaz_v1:soc_ioctl.obj
 0001:00006e68       ??_C@_1GE@OEJKKMF@?$AAW?$AAA?$AAR?$AAN?$AA?3?$AA?5?$AAI?$AAO?$AAC?$AAT?$AAL?$AA_?$AAH?$AAA?$AAL?$AA_?$AAF?$AAO?$AAR?$AAC?$AAE?$AA_?$AAI?$AAR?$AAQ?$AA?5?$AAi?$AAn?$AAv?$AAa?$AAl?$AAi@ 00017e68     oal_ioctl_mx25_topaz_v1:soc_ioctl.obj
 0001:00006ed0       ??_C@_1FO@LEIDEBNM@?$AAW?$AAA?$AAR?$AAN?$AA?3?$AA?5?$AAI?$AAO?$AAC?$AAT?$AAL?$AA_?$AAH?$AAA?$AAL?$AA_?$AAF?$AAO?$AAR?$AAC?$AAE?$AA_?$AAI?$AAR?$AAQ?$AA?5?$AAi?$AAn?$AAv?$AAa?$AAl?$AAi@ 00017ed0     oal_ioctl_mx25_topaz_v1:soc_ioctl.obj
 0001:00006f30       ??_C@_1CO@CKJKOMNN@?$AA?$CL?$AAO?$AAA?$AAL?$AAI?$AAo?$AAC?$AAt?$AAl?$AAH?$AAa?$AAl?$AAF?$AAo?$AAr?$AAc?$AAe?$AAI?$AAr?$AAq?$AA?$AN?$AA?6?$AA?$AA@ 00017f30     oal_ioctl_mx25_topaz_v1:soc_ioctl.obj
 0001:00006f60       ??_C@_1EE@MIMADDNP@?$AA?$CL?$AAO?$AAA?$AAL?$AAI?$AAo?$AAC?$AAt?$AAl?$AAH?$AAa?$AAl?$AAU?$AAn?$AAf?$AAo?$AAr?$AAc?$AAe?$AAI?$AAr?$AAq?$AA?$CI?$AAr?$AAc?$AA?5?$AA?$DN?$AA?5?$AA?$CF?$AAd?$AA?$CJ?$AA?$AN@ 00017f60     oal_ioctl_mx25_topaz_v1:soc_ioctl.obj
 0001:00006fa8       ??_C@_1GI@MPFODPCJ@?$AAW?$AAA?$AAR?$AAN?$AA?3?$AA?5?$AAI?$AAO?$AAC?$AAT?$AAL?$AA_?$AAH?$AAA?$AAL?$AA_?$AAU?$AAN?$AAF?$AAO?$AAR?$AAC?$AAE?$AA_?$AAI?$AAR?$AAQ?$AA?5?$AAi?$AAn?$AAv?$AAa@ 00017fa8     oal_ioctl_mx25_topaz_v1:soc_ioctl.obj
 0001:00007010       ??_C@_1GC@CENCNJJG@?$AAW?$AAA?$AAR?$AAN?$AA?3?$AA?5?$AAI?$AAO?$AAC?$AAT?$AAL?$AA_?$AAH?$AAA?$AAL?$AA_?$AAU?$AAN?$AAF?$AAO?$AAR?$AAC?$AAE?$AA_?$AAI?$AAR?$AAQ?$AA?5?$AAi?$AAn?$AAv?$AAa@ 00018010     oal_ioctl_mx25_topaz_v1:soc_ioctl.obj
 0001:00007074       ??_C@_1DC@MDJDDFNJ@?$AA?$CL?$AAO?$AAA?$AAL?$AAI?$AAo?$AAC?$AAt?$AAl?$AAH?$AAa?$AAl?$AAU?$AAn?$AAf?$AAo?$AAr?$AAc?$AAe?$AAI?$AAr?$AAq?$AA?$AN?$AA?6?$AA?$AA@ 00018074     oal_ioctl_mx25_topaz_v1:soc_ioctl.obj
 0001:00007138       ??_C@_1EI@MCIJGMLN@?$AA?9?$AAO?$AAA?$AAL?$AAI?$AAo?$AAC?$AAt?$AAl?$AAH?$AAa?$AAl?$AAG?$AAe?$AAt?$AAH?$AAW?$AAE?$AAn?$AAt?$AAr?$AAo?$AAp?$AAy?$AA?$CI?$AAr?$AAc?$AA?5?$AA?$DN?$AA?5?$AA?$CF?$AAd@ 00018138     oal_ioctl_mx25_topaz_v1:hwentropy.obj
 0001:00007180       ??_C@_1GE@KDBGDMBH@?$AAW?$AAA?$AAR?$AAN?$AA?3?$AA?5?$AAO?$AAA?$AAL?$AAI?$AAo?$AAC?$AAt?$AAl?$AAH?$AAa?$AAl?$AAG?$AAe?$AAt?$AAH?$AAW?$AAE?$AAn?$AAt?$AAr?$AAo?$AAp?$AAy?$AA?3?$AA?5?$AAB@ 00018180     oal_ioctl_mx25_topaz_v1:hwentropy.obj
 0001:00007278       ??_C@_1KO@FKDDMANO@?$AAC?$AA?3?$AA?2?$AAW?$AAI?$AAN?$AAC?$AAE?$AAR?$AAO?$AAO?$AAT?$AAS?$AA?2?$AAT?$AAo?$AAp?$AAa?$AAz?$AA?2?$AAW?$AAI?$AAN?$AAC?$AAE?$AA6?$AA0?$AA0?$AA?2?$AAP?$AAL?$AAA@ 00018278     cspiutils_oal:cspiutils_oal.obj
 0001:000073b8       ??_C@_1EI@PJAHKOP@?$AA?9?$AAO?$AAA?$AAL?$AAI?$AAo?$AAc?$AAt?$AAl?$AAH?$AAa?$AAl?$AAG?$AAe?$AAt?$AAC?$AAa?$AAc?$AAh?$AAe?$AAI?$AAn?$AAf?$AAo?$AA?$CI?$AAr?$AAc?$AA?5?$AA?$DN?$AA?5?$AA?$CF?$AAd@ 000183b8     oal_cache_arm926:ioctl.obj
 0001:00007400       ??_C@_1GE@MBKHJMBD@?$AAW?$AAA?$AAR?$AAN?$AA?3?$AA?5?$AAO?$AAA?$AAL?$AAI?$AAo?$AAc?$AAt?$AAl?$AAH?$AAa?$AAl?$AAG?$AAe?$AAt?$AAC?$AAa?$AAc?$AAh?$AAe?$AAI?$AAn?$AAf?$AAo?$AA?3?$AA?5?$AAB@ 00018400     oal_cache_arm926:ioctl.obj
 0001:00007468       ??_C@_1HM@KKNPJOOC@?$AAW?$AAA?$AAR?$AAN?$AA?3?$AA?5?$AAO?$AAA?$AAL?$AAI?$AAo?$AAc?$AAt?$AAl?$AAH?$AAa?$AAl?$AAG?$AAe?$AAt?$AAC?$AAa?$AAc?$AAh?$AAe?$AAI?$AAn?$AAf?$AAo?$AA?3?$AA?5?$AAI@ 00018468     oal_cache_arm926:ioctl.obj
 0001:000074e8       ??_C@_1EA@GDPMLOAC@?$AA?$CL?$AAO?$AAA?$AAL?$AAI?$AAo?$AAc?$AAt?$AAl?$AAH?$AAa?$AAl?$AAG?$AAe?$AAt?$AAC?$AAa?$AAc?$AAh?$AAe?$AAI?$AAn?$AAf?$AAo?$AA?$CI?$AA?4?$AA?4?$AA?4?$AA?$CJ?$AA?$AN?$AA?6?$AA?$AA@ 000184e8     oal_cache_arm926:ioctl.obj
 0001:000075b8       ??_C@_1EI@JAFAIJEH@?$AA?$CL?$AAO?$AAA?$AAL?$AAI?$AAo?$AAC?$AAt?$AAl?$AAH?$AAa?$AAl?$AAG?$AAe?$AAt?$AAH?$AAW?$AAE?$AAn?$AAt?$AAr?$AAo?$AAp?$AAy?$AA?$CI?$AAr?$AAc?$AA?5?$AA?$DN?$AA?5?$AA?$CF?$AAd@ 000185b8     oal_oemioctrl_common_topaz_v1:ioctrl.obj
 0001:00007620       PaFromVa                   00018620 f   nkldr:armstart.obj
 0001:00007670       VaFromPa                   00018670 f   nkldr:armstart.obj
 0001:000076bc       GetCpuId                   000186bc f   nkldr:armstart.obj
 0001:000076c4       KernelStart                000186c4 f   nkldr:armstart.obj
 0001:000078cc       ARMInit                    000188cc f   nkldr:arminit.obj
 0001:00007944       KernelRelocate             00018944 f   nkldr:ldrcmn.obj
 0001:00007a4c       FindKernelEntry            00018a4c f   nkldr:ldrcmn.obj
 0001:00007b3c       SetOsAxsDataBlockPointer   00018b3c f   nkldr:kdinfo.obj
 0001:00007b78       _stricmp                   00018b78 f   nkldr:strings.obj
 0001:00007c10       memset                     00018c10 f   fulllibc:memset.obj
 0001:00007c98       memcpy                     00018c98 f   fulllibc:memcpy.obj
 0001:00008044       memcpybigblk               00019044 f   fulllibc:memcpy.obj
 0001:000089f8       tolower                    000199f8 f   fulllibc:tolower.obj
 0001:00008abc       OEMInitGlobals             00019abc f   oemmain:oemglobal.obj
 0001:00008b18       NKOutputDebugString        00019b18 f   nkstub:nkstub.obj
 0001:00008b4c       NKvDbgPrintfW              00019b4c f   nkstub:nkstub.obj
 0001:00008b84       NKDbgPrintfW               00019b84 f   nkstub:nkstub.obj
 0001:00008bd8       NKwvsprintfW               00019bd8 f   nkstub:nkstub.obj
 0001:00008c30       NKSetLastError             00019c30 f   nkstub:nkstub.obj
 0001:00008c64       NKGetLastError             00019c64 f   nkstub:nkstub.obj
 0001:00008ca4       EnterCriticalSection       00019ca4 f   nkstub:nkstub.obj
 0001:00008cd8       LeaveCriticalSection       00019cd8 f   nkstub:nkstub.obj
 0001:00008d0c       InitializeCriticalSection  00019d0c f   nkstub:nkstub.obj
 0001:00008d40       DeleteCriticalSection      00019d40 f   nkstub:nkstub.obj
 0001:00008d74       INTERRUPTS_OFF             00019d74 f   nkstub:nkstub.obj
 0001:00008d9c       INTERRUPTS_ON              00019d9c f   nkstub:nkstub.obj
 0001:00008dc4       INTERRUPTS_ENABLE          00019dc4 f   nkstub:nkstub.obj
 0001:00008e10       HookInterrupt              00019e10 f   nkstub:nkstub.obj
 0001:00008e60       UnhookInterrupt            00019e60 f   nkstub:nkstub.obj
 0001:00008eb0       NKCallIntChain             00019eb0 f   nkstub:nkstub.obj
 0001:00008efc       NKIsSysIntrValid           00019efc f   nkstub:nkstub.obj
 0001:00008f48       NKSetInterruptEvent        00019f48 f   nkstub:nkstub.obj
 0001:00008f94       NKSleep                    00019f94 f   nkstub:nkstub.obj
 0001:00008fc8       NKVirtualSetAttributes     00019fc8 f   nkstub:nkstub.obj
 0001:00009028       NKCreateStaticMapping      0001a028 f   nkstub:nkstub.obj
 0001:00009078       NKDeleteStaticMapping      0001a078 f   nkstub:nkstub.obj
 0001:000090c8       NKRegCloseKey              0001a0c8 f   nkstub:nkstub.obj
 0001:00009114       NKRegFlushKey              0001a114 f   nkstub:nkstub.obj
 0001:00009160       NKRegCreateKeyExW          0001a160 f   nkstub:nkstub.obj
 0001:000091e0       NKRegOpenKeyExW            0001a1e0 f   nkstub:nkstub.obj
 0001:00009240       NKRegQueryValueExW         0001a240 f   nkstub:nkstub.obj
 0001:000092a8       NKRegSetValueExW           0001a2a8 f   nkstub:nkstub.obj
 0001:00009310       NKForceCleanBoot           0001a310 f   nkstub:nkstub.obj
 0001:00009338       NKReboot                   0001a338 f   nkstub:nkstub.obj
 0001:00009384       NKwcslen                   0001a384 f   nkstub:nkstub.obj
 0001:000093d0       NKwcscmp                   0001a3d0 f   nkstub:nkstub.obj
 0001:00009420       NKwcsicmp                  0001a420 f   nkstub:nkstub.obj
 0001:00009470       NKwcsnicmp                 0001a470 f   nkstub:nkstub.obj
 0001:000094c4       NKwcscpy                   0001a4c4 f   nkstub:nkstub.obj
 0001:000094fc       NKwcsncpy                  0001a4fc f   nkstub:nkstub.obj
 0001:00009550       NKstrcmpiAandW             0001a550 f   nkstub:nkstub.obj
 0001:000095a0       NKUnicodeToAscii           0001a5a0 f   nkstub:nkstub.obj
 0001:000095dc       NKAsciiToUnicode           0001a5dc f   nkstub:nkstub.obj
 0001:00009618       NKSystemTimeToFileTime     0001a618 f   nkstub:nkstub.obj
 0001:00009668       NKFileTimeToSystemTime     0001a668 f   nkstub:nkstub.obj
 0001:000096b8       NKCompareFileTime          0001a6b8 f   nkstub:nkstub.obj
 0001:00009710       ProfilerHit                0001a710 f   nkstub:nkstub.obj
 0001:00009774       ProfilerHitEx              0001a774 f   nkstub:nkstub.obj
 0001:000097a8       GetEPC                     0001a7a8 f   nkstub:nkstub.obj
 0001:000097e8       NKPhysToVirt               0001a7e8 f   nkstub:nkstub.obj
 0001:00009838       NKVirtToPhys               0001a838 f   nkstub:nkstub.obj
 0001:00009884       __GetUserKData             0001a884 f   nkstub:nkstub.obj
 0001:000098b4       __report_gsfailure         0001a8b4 f   nkstub:nkstub.obj
 0001:000098dc       GetOriginalDAbortHandlerAddress 0001a8dc f   nkstub:nkstub.obj
 0001:0000990c       NKSetDataAbortHandler      0001a90c f   nkstub:nkstub.obj
 0001:00009998       OEMHaltSystem              0001a998 f   oal:init.obj
 0001:0000999c       OEMInit                    0001a99c f   oal:init.obj
 0001:0000a5b0       RNGB_Init                  0001b5b0 f   oal:rngb.obj
 0001:0000a760       OALIoCtlHalGetRandomSeed   0001b760 f   oal:rngb.obj
 0001:0000a7d4       RNGB_GetRandomData         0001b7d4 f   oal:rngb.obj
 0001:0000a9c4       OALPmicInit                0001b9c4 f   oal:pmic.obj
 0001:0000aa2c       OALTimerNotifyReschedule   0001ba2c f   oal:timer.obj
 0001:0000ad80       OALTimerGetClkSrc          0001bd80 f   oal:timer.obj
 0001:0000adb4       OALTimerGetClkPrescalar    0001bdb4 f   oal:timer.obj
 0001:0000adcc       OALTimerGetClkFreq         0001bdcc f   oal:timer.obj
 0001:0000aed8       OALCPUIdle                 0001bed8 f   oal:timer.obj
 0001:0000aee4       WdogService                0001bee4 f   oal:timer.obj
 0001:0000af84       WdogInit                   0001bf84 f   oal:timer.obj
 0001:0000b0ac       RefreshWatchdogTimer       0001c0ac f   oal:timer.obj
 0001:0000b1bc       InitWatchDogTimer          0001c1bc f   oal:timer.obj
 0001:0000b264       OALCPUEnterWFI             0001c264 f   oal:wfi.obj
 0001:0000b270       OEMGetTickCount            0001c270 f   oal_timer_epit_common_topaz_v1:timer.obj
 0001:0000b350       OALTimerQueryPerformanceCounter 0001c350 f   oal_timer_epit_common_topaz_v1:timer.obj
 0001:0000b430       OALTimerQueryPerformanceFrequency 0001c430 f   oal_timer_epit_common_topaz_v1:timer.obj
 0001:0000b4c0       OALTimerUpdateRescheduleTime 0001c4c0 f   oal_timer_epit_common_topaz_v1:timer.obj
 0001:0000b638       OALTimerInit               0001c638 f   oal_timer_epit_common_topaz_v1:timer.obj
 0001:0000bb94       OALTimerIntrHandler        0001cb94 f   oal_timer_epit_common_topaz_v1:timer.obj
 0001:0000be20       OALTimerCountsSinceSysTick 0001ce20 f   oal_timer_epit_common_topaz_v1:timer.obj
 0001:0000be58       OEMIdle                    0001ce58 f   oal_timer_epit_common_topaz_v1:timer.obj
 0001:0000bf5c       OALTimerSetCompare         0001cf5c f   oal_timer_epit_common_topaz_v1:timer.obj
 0001:0000bf9c       OALTimerRecharge           0001cf9c f   oal_timer_epit_common_topaz_v1:timer.obj
 0001:0000c028       OALTimerGetIrq             0001d028 f   oal_timer_epit_mx25_topaz_v1:soc_timer.obj
 0001:0000c040       OALTimerGetBaseRegAddr     0001d040 f   oal_timer_epit_mx25_topaz_v1:soc_timer.obj
 0001:0000c05c       OEMInterruptHandlerFIQ     0001d05c f   oal_intr_mx25_topaz_v1:fiq.obj
 0001:0000c060       OALIntrInit                0001d060 f   oal_intr_mx25_topaz_v1:intr.obj
 0001:0000c494       OALIntrRequestIrqs         0001d494 f   oal_intr_mx25_topaz_v1:intr.obj
 0001:0000d228       OALIntrEnableIrqs          0001e228 f   oal_intr_mx25_topaz_v1:intr.obj
 0001:0000d4f8       OALIntrDisableIrqs         0001e4f8 f   oal_intr_mx25_topaz_v1:intr.obj
 0001:0000d75c       OALIntrDoneIrqs            0001e75c f   oal_intr_mx25_topaz_v1:intr.obj
 0001:0000d9cc       OEMInterruptHandler        0001e9cc f   oal_intr_mx25_topaz_v1:intr.obj
 0001:0000ddec       OALIntrMapInit             0001edec f   oal_intr_mx25_topaz_v1:map.obj
 0001:0000df48       OALIntrStaticTranslate     0001ef48 f   oal_intr_mx25_topaz_v1:map.obj
 0001:0000e0b8       OALIntrTranslateSysIntr    0001f0b8 f   oal_intr_mx25_topaz_v1:map.obj
 0001:0000e1b4       OALIntrTranslateIrq        0001f1b4 f   oal_intr_mx25_topaz_v1:map.obj
 0001:0000e298       OALIntrRequestSysIntr      0001f298 f   oal_intr_mx25_topaz_v1:map.obj
 0001:0000e918       OALIntrReleaseSysIntr      0001f918 f   oal_intr_mx25_topaz_v1:map.obj
 0001:0000eb3c       OEMInterruptEnable         0001fb3c f   oal_intr_mx25_topaz_v1:map.obj
 0001:0000ec8c       OEMInterruptDisable        0001fc8c f   oal_intr_mx25_topaz_v1:map.obj
 0001:0000ed90       OEMInterruptMask           0001fd90 f   oal_intr_mx25_topaz_v1:map.obj
 0001:0000eec4       OEMInterruptDone           0001fec4 f   oal_intr_mx25_topaz_v1:map.obj
 0001:0000efc8       OEMIoControl               0001ffc8 f   oal_ioctl_mx25_topaz_v1:ioctl.obj
 0001:0000f298       OEMPowerOff                00020298 f   oal_power_mx25_topaz_v1:off.obj
 0001:0000f828       OALClockSetGatingMode      00020828 f   oal_power_mx25_topaz_v1:off.obj
 0001:0000f8d4       OALInitializeClockGating   000208d4 f   oal_power_mx25_topaz_v1:off.obj
 0001:0000fd4c       OALPowerWakeSource         00020d4c f   oal_power_mx25_topaz_v1:ioctl.obj
 0001:0000fdc0       OALIoCtlHalEnableWake      00020dc0 f   oal_power_mx25_topaz_v1:ioctl.obj
 0001:0000ff80       OALIoCtlHalDisableWake     00020f80 f   oal_power_mx25_topaz_v1:ioctl.obj
 0001:00010144       OALIoCtlHalGetWakeSource   00021144 f   oal_power_mx25_topaz_v1:ioctl.obj
 0001:00010280       OEMSetAlarmTime            00021280 f   oal_RTC_mx25_topaz_v1:alarm.obj
 0001:00010610       DRYICE_WRITE               00021610 f   oal_RTC_mx25_topaz_v1:rtc.obj
 0001:00010648       DRYICE_READ                00021648 f   oal_RTC_mx25_topaz_v1:rtc.obj
 0001:0001068c       OALRtcMap                  0002168c f   oal_RTC_mx25_topaz_v1:rtc.obj
 0001:000107a8       OALInitRTC                 000217a8 f   oal_RTC_mx25_topaz_v1:rtc.obj
 0001:000109a0       OALIoCtlHalInitRTC         000219a0 f   oal_RTC_mx25_topaz_v1:rtc.obj
 0001:00010b84       OEMGetRealTime             00021b84 f   oal_RTC_mx25_topaz_v1:rtc.obj
 0001:00010dec       OEMSetRealTime             00021dec f   oal_RTC_mx25_topaz_v1:rtc.obj
 0001:00011198       OALPAtoVA                  00022198 f   oal_memory_arm:memory.obj
 0001:000112c0       OALVAtoPA                  000222c0 f   oal_memory_arm:memory.obj
 0001:000113f8       OEMProfileTimerEnable      000223f8 f   oal_profiler_gpt_mx25_topaz_v1:profiler.obj
 0001:000115cc       OEMProfileTimerDisable     000225cc f   oal_profiler_gpt_mx25_topaz_v1:profiler.obj
 0001:0001168c       OALProfileIntrHandler      0002268c f   oal_profiler_gpt_mx25_topaz_v1:profiler.obj
 0001:000116ec       OALProfileGetIrq           000226ec f   oal_profiler_gpt_mx25_topaz_v1:soc_profiler.obj
 0001:00011704       OALProfileGetBaseRegAddr   00022704 f   oal_profiler_gpt_mx25_topaz_v1:soc_profiler.obj
 0001:00011720       OALProfileTimerEnable      00022720 f   oal_profiler_gpt_mx25_topaz_v1:soc_profiler.obj
 0001:00011738       OALProfileTimerDisable     00022738 f   oal_profiler_gpt_mx25_topaz_v1:soc_profiler.obj
 0001:00011750       OEMGetExtensionDRAM        00022750 f   oal_other:memory.obj
 0001:00011778       OEMWriteDebugString        00022778 f   oal_other:debug.obj
 0001:000117cc       OALLogSetZones             000227cc f   oal_log:debug.obj
 0001:00011838       OALLogSerial               00022838 f   oal_log:log.obj
 0001:00011894       OALLogPrintf               00022894 f   oal_log:log.obj
 0001:000118d0       OALIsProcessorFeaturePresent 000228d0 f   oal_misc_arm:feature.obj
 0001:00011a38       OALGetIdCode               00022a38 f   oal_misc_arm:getidcode.obj
 0001:00011a40       __GSHandlerCheck           00022a40 f   fulllibc:gshandler.obj
 0001:00011a88       __GSHandlerCheckCommon     00022a88 f   fulllibc:gshandler.obj
 0001:00011b30       __security_check_cookie    00022b30 f   fulllibc:armsecgs.obj
 0001:00011b44       __gsfailure                00022b44 f   fulllibc:armsecgs.obj
 0001:00011b88       __rt_udiv                  00022b88 f   fulllibc:__udiv.obj
 0001:00011c4c       __rt_udivrem64by64         00022c4c f   fulllibc:mdsdiv64.obj
 0001:00011d44       __rt_divrem64by64          00022d44 f   fulllibc:mdsdiv64.obj
 0001:00011d94       __rt_udiv64by64            00022d94 f   fulllibc:mdsdiv64.obj
 0001:00011da4       __rt_urem64by64            00022da4 f   fulllibc:mdsdiv64.obj
 0001:00011dbc       __rt_sdiv64by64            00022dbc f   fulllibc:mdsdiv64.obj
 0001:00011dcc       __rt_srem64by64            00022dcc f   fulllibc:mdsdiv64.obj
 0001:00011de4       __rt_sdiv                  00022de4 f   fulllibc:__div.obj
 0001:00011ec0       __raise_int_divide_by_zero 00022ec0 f   fulllibc:diverr.obj
 0001:00011ee4       __raise_int_overflow       00022ee4 f   fulllibc:diverr.obj
 0001:00011f08       __crtRaiseException        00022f08 f   fulllibc:raiseexc.obj
 0001:00011f3c       OALSerialInit              00022f3c f   bspcmn:debugserial.obj
 0001:00011fb8       OEMInitDebugSerial         00022fb8 f   bspcmn:debugserial.obj
 0001:000121e4       OEMWriteDebugByte          000231e4 f   bspcmn:debugserial.obj
 0001:00012240       OEMReadDebugByte           00023240 f   bspcmn:debugserial.obj
 0001:00012290       OEMWriteDebugLED           00023290 f   bspcmn:debugserial.obj
 0001:000122a4       OALBspArgsInit             000232a4 f   bspcmn:bspargs.obj
 0001:00012a7c       OALBspArgsPrint            00023a7c f   bspcmn:bspargs.obj
 0001:00013004       OALConfigSerialUART        00024004 f   serialutils:serialutils.obj
 0001:00013448       OALConfigSerialIOMUX       00024448 f   serialutils:serialutils.obj
 0001:00013548       OALArgsQuery               00024548 f   args:args.obj
 0001:00013884       PmicOpen                   00024884 f   pmicutils:mc34704utils.obj
 0001:000138b0       PmicClose                  000248b0 f   pmicutils:mc34704utils.obj
 0001:000138b4       PmicEnable                 000248b4 f   pmicutils:mc34704utils.obj
 0001:000138f0       PmicEnDSMVoltage           000248f0 f   pmicutils:mc34704utils.obj
 0001:0001393c       PmicDisDSMVoltage          0002493c f   pmicutils:mc34704utils.obj
 0001:00013988       PmicEnableExternal3V3      00024988 f   pmicutils:mc34704utils.obj
 0001:00013a0c       PmicRegulatorSetVoltageLevel 00024a0c f   pmicutils:mc34704utils.obj
 0001:00013b74       PmicRegulatorGetVoltageLevel 00024b74 f   pmicutils:mc34704utils.obj
 0001:00013ba8       PmicSetRegister            00024ba8 f   pmicutils:mc34704utils.obj
 0001:00013c94       PmicGetRegister            00024c94 f   pmicutils:mc34704utils.obj
 0001:00013ec0       OALI2cInit                 00024ec0 f   i2cutils:i2cutils.obj
 0001:000140f0       OALI2cEnable               000250f0 f   i2cutils:i2cutils.obj
 0001:000141c0       OALI2cDisable              000251c0 f   i2cutils:i2cutils.obj
 0001:000141f8       OALI2cCalculateClkRateDiv  000251f8 f   i2cutils:i2cutils.obj
 0001:00014504       OALI2cGenerateStart        00025504 f   i2cutils:i2cutils.obj
 0001:000147d4       OALI2cRepeatedStart        000257d4 f   i2cutils:i2cutils.obj
 0001:00014a34       OALI2cWriteData            00025a34 f   i2cutils:i2cutils.obj
 0001:00014cd8       OALI2cReadData             00025cd8 f   i2cutils:i2cutils.obj
 0001:00014fd4       OALI2cSetReceiveMode       00025fd4 f   i2cutils:i2cutils.obj
 0001:00015060       OALI2cSetTxAck             00026060 f   i2cutils:i2cutils.obj
 0001:000150ec       OALI2cPutData              000260ec f   i2cutils:i2cutils.obj
 0001:0001535c       OALI2cGetData              0002635c f   i2cutils:i2cutils.obj
 0001:00015558       OALI2cGenerateStop         00026558 f   i2cutils:i2cutils.obj
 0001:000157d4       OEMCacheRangeFlush         000267d4 f   oal_cache_arm926:flush.obj
 0001:00015aa0       OEMARMCacheMode            00026aa0 f   oal_cache_arm926:cachemode.obj
 0001:00015aa8       OALCacheGlobalsInit        00026aa8 f   oal_cache_arm926:init.obj
 0001:00015c20       OALClearDTLB               00026c20 f   oal_cache_arm926:cleardtlb.obj
 0001:00015c2c       OALClearDTLBEntry          00026c2c f   oal_cache_arm926:cleardtlbentry.obj
 0001:00015c34       OALClearITLB               00026c34 f   oal_cache_arm926:clearitlb.obj
 0001:00015c40       OALClearITLBEntry          00026c40 f   oal_cache_arm926:clearitlbentry.obj
 0001:00015c48       OALFlushICacheLines        00026c48 f   oal_cache_arm926:flushiclines.obj
 0001:00015c68       OALFlushICache             00026c68 f   oal_cache_arm926:flushic.obj
 0001:00015c74       OALCleanDCacheLines        00026c74 f   oal_cache_arm926:cleandclines.obj
 0001:00015c9c       OALCleanDCache             00026c9c f   oal_cache_arm926:cleandc.obj
 0001:00015ca8       OALFlushDCacheLines        00026ca8 f   oal_cache_arm926:flushdclines.obj
 0001:00015cc8       OALFlushDCache             00026cc8 f   oal_cache_arm926:flushdc.obj
 0001:00015cd4       KITLIoctl                  00026cd4 f   nkstub:kitlstub.obj
 0001:00015d3c       BSPIntrInit                00026d3c f   oal:intr.obj
 0001:00015d54       BSPIntrRequestIrqs         00026d54 f   oal:intr.obj
 0001:00015e50       BSPIntrEnableIrq           00026e50 f   oal:intr.obj
 0001:00015f00       BSPIntrDisableIrq          00026f00 f   oal:intr.obj
 0001:00015fb0       BSPIntrDoneIrq             00026fb0 f   oal:intr.obj
 0001:00016060       BSPIntrActiveIrq           00027060 f   oal:intr.obj
 0001:00016110       OALIoCtlHalPostInit        00027110 f   oal:ioctl.obj
 0001:00016144       OALIoCtlHalPresuspend      00027144 f   oal:ioctl.obj
 0001:00016168       OALIoCtlHalGetHiveCleanFlag 00027168 f   oal:ioctl.obj
 0001:000161d0       OALIoCtlHalInitRegistry    000271d0 f   oal:ioctl.obj
 0001:000167e0       OALIoCtlQueryDispSettings  000277e0 f   oal:ioctl.obj
 0001:000168f4       OALIoCtlQuerySiVersion     000278f4 f   oal:ioctl.obj
 0001:000169f0       OALIoCtlSharedCspiTransfer 000279f0 f   oal:ioctl.obj
 0001:00016b78       CspiBufRd8                 00027b78 f   oal:ioctl.obj
 0001:00016ba8       CspiBufRd16                00027ba8 f   oal:ioctl.obj
 0001:00016bd8       CspiBufRd32                00027bd8 f   oal:ioctl.obj
 0001:00016c08       CspiBufWrt8                00027c08 f   oal:ioctl.obj
 0001:00016c38       CspiBufWrt16               00027c38 f   oal:ioctl.obj
 0001:00016c6c       CspiBufWrt32               00027c6c f   oal:ioctl.obj
 0001:00017214       DumpCspiRegs               00028214 f   oal:ioctl.obj
 0001:000172ec       OALCPUPowerOff             000282ec f   oal:power.obj
 0001:000174a8       BSPPowerOff                000284a8 f   oal:power.obj
 0001:000174e8       BSPPowerOn                 000284e8 f   oal:power.obj
 0001:00017528       OALProfileGetClkSrc        00028528 f   oal:profiler.obj
 0001:00017540       OALProfileGetClkFreq       00028540 f   oal:profiler.obj
 0001:00017608       OALIoCtlHalDdkCall         00028608 f   oal_io:ioctl.obj
 0001:00017c04       OALIoBusPowerOff           00028c04 f   oal_io:power.obj
 0001:00017cc4       OALIoBusPowerOn            00028cc4 f   oal_io:power.obj
 0001:00017d84       OALIoTransBusAddress       00028d84 f   oal_io:trans.obj
 0001:00017ed0       OALIoTransSystemAddress    00028ed0 f   oal_io:trans.obj
 0001:00017fd0       OALIoReadBusData           00028fd0 f   oal_io:data.obj
 0001:00018000       OALIoWriteBusData          00029000 f   oal_io:data.obj
 0001:00018030       OALIoCtlHalRequestSysIntr  00029030 f   oal_intr_mx25_topaz_v1:ioctl.obj
 0001:00018390       OALIoCtlHalReleaseSysIntr  00029390 f   oal_intr_mx25_topaz_v1:ioctl.obj
 0001:000184cc       OALIoCtlHalRequestIrq      000294cc f   oal_intr_mx25_topaz_v1:ioctl.obj
 0001:0001866c       OALIoCtlHalUpdateMode      0002966c f   oal_ioctl_mx25_topaz_v1:imgupd.obj
 0001:00018788       OALIoCtlHalGetRegSecureKeys 00029788 f   oal_ioctl_mx25_topaz_v1:securekeys.obj
 0001:00018868       OALIoCtlProcessorInfo      00029868 f   oal_ioctl_mx25_topaz_v1:procinfo.obj
 0001:00018ba0       OALIoCtlHalGetUUID         00029ba0 f   oal_ioctl_mx25_topaz_v1:uuid.obj
 0001:00018da0       OALIoCtlHalGetDeviceInfo   00029da0 f   oal_ioctl_mx25_topaz_v1:deviceinfo.obj
 0001:00019860       OALIoCtlHalGetDeviceId     0002a860 f   oal_ioctl_mx25_topaz_v1:deviceid.obj
 0001:00019c28       OALIoCtlHalReboot          0002ac28 f   oal_ioctl_mx25_topaz_v1:reboot.obj
 0001:00019c94       OALIoCtlGetResetCause      0002ac94 f   oal_ioctl_mx25_topaz_v1:reboot.obj
 0001:00019d10       OALIoCtlHalIrq2Sysintr     0002ad10 f   oal_ioctl_mx25_topaz_v1:soc_ioctl.obj
 0001:00019e70       OALIoCtlHalForceIrq        0002ae70 f   oal_ioctl_mx25_topaz_v1:soc_ioctl.obj
 0001:0001a058       OALIoCtlHalUnforceIrq      0002b058 f   oal_ioctl_mx25_topaz_v1:soc_ioctl.obj
 0001:0001a244       OALIoCtlHalGetHWEntropy    0002b244 f   oal_ioctl_mx25_topaz_v1:hwentropy.obj
 0001:0001a344       __C_specific_handler       0002b344 f   fulllibc:chandler.obj
 0001:0001a6b4       strlen                     0002b6b4 f   fulllibc:mdsstrlen.obj
 0001:0001a718       __C_ExecuteTerminationHandler 0002b718 f   fulllibc:jmpuwind.obj
 0001:0001a718       __C_ExecuteExceptionFilter 0002b718 f   fulllibc:jmpuwind.obj
 0001:0001a758       CSPIRequest                0002b758 f   cspiutils_oal:cspiutils_oal.obj
 0001:0001a8b4       CSPIRelease                0002b8b4 f   cspiutils_oal:cspiutils_oal.obj
 0001:0001a938       OALIoCtlHalGetCacheInfo    0002b938 f   oal_cache_arm926:ioctl.obj
 0001:0001abc8       OALIoCtlKitlGetInfo        0002bbc8 f   oal_oemioctrl_common_topaz_v1:ioctrl.obj
 0001:0001ad3c       InterlockedExchange        0002bd3c f   nkstub:intrlock.obj
 0001:0001ad44       InterlockedTestExchange    0002bd44 f   nkstub:intrlock.obj
 0001:0001ad50       InterlockedCompareExchange 0002bd50 f   nkstub:intrlock.obj
 0001:0001ad58       InterlockedExchangeAdd     0002bd58 f   nkstub:intrlock.obj
 0001:0001ad60       InterlockedIncrement       0002bd60 f   nkstub:intrlock.obj
 0001:0001ad80       InterlockedDecrement       0002bd80 f   nkstub:intrlock.obj
 0001:0001ada0       V6_WriteBarrier            0002bda0 f   nkstub:intrlock.obj
 0003:00000000       OsAxsDataBlock_2           00032000     nkldr:kdinfo.obj
 0003:00000080       OsAxsHwTrap                00032080     nkldr:kdinfo.obj
 0003:0000021c       g_pOemGlobal               0003221c     oemmain:oemglobal.obj
 0003:00000220       __security_cookie          00032220     nkstub:nkstub.obj
 0003:00000224       __security_cookie_complement 00032224     nkstub:nkstub.obj
 0003:00000228       g_dwResetCause             00032228     oal:init.obj
 0003:0000022c       dwOEMDrWatsonSize          0003222c     oal:init.obj
 0003:00000238       g_oalWakeSource            00032238     oal_power_mx25_topaz_v1:ioctl.obj
 0003:00000240       initialOALLogZones         00032240     oal_log:debug.obj
 0003:00000248       dpCurSettings              00032248     oal_log:debug.obj
 0003:000006a4       g_oalIoCtlPlatformType     000326a4     oal:ioctl.obj
 0003:000006a8       g_oalIoCtlPlatformOEM      000326a8     oal:ioctl.obj
 0003:000006ac       g_oalIoCtlProcessorVendor  000326ac     oal:ioctl.obj
 0003:000006b0       g_oalIoCtlProcessorName    000326b0     oal:ioctl.obj
 0003:000006b4       g_oalIoCtlProcessorCore    000326b4     oal:ioctl.obj
 0003:000006f0       g_pProfilerISR             000326f0     oal_intr_mx25_topaz_v1:intr.obj
 0003:00000b58       g_bOalPostInit             00032b58     oal:ioctl.obj
 0003:00000b5c       g_oalIoCtlInstructionSet   00032b5c     oal:ioctl.obj
 0003:00000b60       g_oalIoCtlClockSpeed       00032b60     oal:ioctl.obj
 0003:00000b84       g_pNKGlobal                00032b84     <common>
 0003:00000b88       g_UPID                     00032b88     <common>
 0003:00000b90       g_pIIM                     00032b90     <common>
 0003:00000b94       g_SREV                     00032b94     <common>
 0003:00000b98       g_pEPIT                    00032b98     <common>
 0003:00000ba0       g_oalTimer                 00032ba0     <common>
 0003:00000be0       g_oalSysIntr2Irq           00032be0     <common>
 0003:00001060       g_pGPIO3                   00033060     <common>
 0003:00001064       g_pAVIC                    00033064     <common>
 0003:00001068       g_pGPIO2                   00033068     <common>
 0003:0000106c       g_pGPIO1                   0003306c     <common>
 0003:00001070       g_pSDMA                    00033070     <common>
 0003:00001074       g_pGPIO4                   00033074     <common>
 0003:00001078       g_oalRtcOriginTime         00033078     <common>
 0003:00001080       g_oalRtcCS                 00033080     <common>
 0003:00001094       g_oalRtcMaxYear            00033094     <common>
 0003:00001098       g_pDryIce                  00033098     <common>
 0003:0000109c       g_pDdkClkConfig            0003309c     <common>
 0003:000010a0       g_pUART                    000330a0     <common>
 0003:000010a4       g_pIOMUX                   000330a4     <common>
 0003:000010a8       g_pCRM                     000330a8     <common>
 0003:000010ac       g_PBCversion               000330ac     <common>
 0003:000010b0       g_oalPerClkFreq            000330b0     <common>
 0003:000010c0       g_UUID                     000330c0     <common>
 0003:000010d0       g_pBSPArgs                 000330d0     <common>
 0003:000010e0       g_oalCacheInfo             000330e0     <common>

 entry point at        0001:00000000

 Static symbols

 0001:00008a54       ReturnFalse                00019a54 f   oemmain:oemglobal.obj
 0001:00008a6c       ReturnSelf                 00019a6c f   oemmain:oemglobal.obj
 0001:00008a94       FakeCalcPage               00019a94 f   oemmain:oemglobal.obj
 0001:0000f964       OALWakeupInterruptEnable   00020964 f   oal_power_mx25_topaz_v1:off.obj
 0001:00012138       InitGlobals                00023138 f   bspcmn:debugserial.obj
 0001:00016560       inet_ntow                  00027560 f   oal:ioctl.obj
 0001:000166cc       uc2wstr                    000276cc f   oal:ioctl.obj
 0001:00016c98       OALCspiNonDMADataExchange  00027c98 f   oal:ioctl.obj
 0001:000190e4       ?GetPlatformType@@YAHPAXIPAIPAPBG@Z 0002a0e4 f   oal_ioctl_mx25_topaz_v1:deviceinfo.obj
 0001:00019178       ?GetOEMInfo@@YAHPAXIPAIPAPBG@Z 0002a178 f   oal_ioctl_mx25_topaz_v1:deviceinfo.obj
 0001:00019228       ?GetPlatformVersion@@YAHPAXIPAIPAPBG@Z 0002a228 f   oal_ioctl_mx25_topaz_v1:deviceinfo.obj
 0001:000192bc       ?GetProjectName@@YAHPAXIPAIPAPBG@Z 0002a2bc f   oal_ioctl_mx25_topaz_v1:deviceinfo.obj
 0001:00019364       ?GetPlatformName@@YAHPAXIPAIPAPBG@Z 0002a364 f   oal_ioctl_mx25_topaz_v1:deviceinfo.obj
 0001:0001941c       ?GetBootMeName@@YAHPAXIPAIPAPBG@Z 0002a41c f   oal_ioctl_mx25_topaz_v1:deviceinfo.obj
 0001:00019590       ?GetUUID@@YAHPAXIPAIPAPBG@Z 0002a590 f   oal_ioctl_mx25_topaz_v1:deviceinfo.obj
 0001:00019650       ?GetGUIDPattern@@YAHPAXIPAIPAPBG@Z 0002a650 f   oal_ioctl_mx25_topaz_v1:deviceinfo.obj
 0001:000196e4       ?CheckBufferSize@@YAHPBXABIPAI1PBG@Z 0002a6e4 f   oal_ioctl_mx25_topaz_v1:deviceinfo.obj
 0001:000197fc       ?ErrorNotSupported@@YAXPBG@Z 0002a7fc f   oal_ioctl_mx25_topaz_v1:deviceinfo.obj
